:020000040000FA
:04080000F1EF0BF019
:1008100003B276EF05F0F2B494EF05F09EB09CEFD2
:1008200005F09EB2A4EF05F0F2A81AEF04F0F2B2C0
:1008300025EF04F0F2A620EF04F0F2B022EF04F06E
:10084000A0EF0BF0F296F290FF00CD90F2929EA0F6
:100850002FEF04F00101533F2FEF04F0542BAEC1F2
:10086000B2F1AFC1B3F1B0C1B4F1B1C1B5F1AAC138
:10087000AEF1ABC1AFF1ACC1B0F1ADC1B1F1A6C148
:10088000AAF1A7C1ABF1A8C1ACF1A9C1ADF1A2C158
:10089000A6F1A3C1A7F1A4C1A8F1A5C1A9F19EC168
:1008A000A2F19FC1A3F1A0C1A4F1A1C1A5F19AC178
:1008B0009EF19BC19FF19CC1A0F19DC1A1F196C188
:1008C0009AF197C19BF198C19CF199C19DF1CECF4E
:1008D00096F1CFCF97F153C198F154C199F1CF6AF6
:1008E000CE6A0101536B546B9E90CD800FBC0F8E6E
:1008F0000FBA7EEF04F00F8AA0EF0BF00F8C0FBE43
:10090000BAEF04F096C19AF197C19BF198C19CF19E
:1009100099C19DF19AC19EF19BC19FF19CC1A0F12B
:100920009DC1A1F19EC1A2F19FC1A3F1A0C1A4F1FB
:10093000A1C1A5F1A2C1A6F1A3C1A7F1A4C1A8F1CB
:10094000A5C1A9F1A6C1AAF1A7C1ABF1A8C1ACF19B
:10095000A9C1ADF1AAC1AEF1ABC1AFF1ACC1B0F16B
:10096000ADC1B1F1AEC1B2F1AFC1B3F1B0C1B4F13B
:10097000B1C1B5F101015E6B5F6B606B616B96514C
:100980005E2797515F2398516023995161239A51B3
:100990005E279B515F239C5160239D5161239E5193
:1009A0005E279F515F23A0516023A1516123A25173
:1009B0005E27A3515F23A4516023A5516123A65153
:1009C0005E27A7515F23A8516023A9516123AA5133
:1009D0005E27AB515F23AC516023AD516123AE5113
:1009E0005E27AF515F23B0516023B1516123B251F3
:1009F0005E27B3515F23B4516023B5516123D89072
:100A00000101613360335F335E33D890010161339C
:100A100060335F335E33D8900101613360335F33FD
:100A20005E3300C10CF101C10DF102C10EF103C131
:100A30000FF104C110F105C111F106C112F107C196
:100A400013F108C114F109C115F10AC116F10BC166
:100A500017F134C135F111B839EF05F00101620E1B
:100A6000046F010E056F000E066F000E076F42EF58
:100A700005F00101A70E046F020E056F000E066F50
:100A8000000E076F5EC100F15FC101F160C102F1AC
:100A900061C103F132EC35F003BF04D018BE02D0BF
:100AA00018A0108C11A05AEF05F010BA5AEF05F0FB
:100AB0000F80108A0CC100F10DC101F10EC102F1CD
:100AC0000FC103F110C104F111C105F112C106F10A
:100AD00013C107F114C108F115C109F116C10AF1DA
:100AE00017C10BF135C134F1A0EF0BF00392ABB29B
:100AF000AB98AB88030103EE00F080517F0BE92631
:100B000004C0EFFF802B8151805D700BD8A48B82D5
:100B100000008051815D700BD8A48B9281518019A7
:100B2000D8B40790A0EF0BF0F2940101453FA0EF7D
:100B30000BF0462BA0EF0BF09E900101533FA0EF6E
:100B40000BF0542BA0EF0BF09E9211B873EF08F04E
:100B5000040066A1ACEF05F08BB4B6EF05F010AC65
:100B6000B6EF05F08B84109CB7EF05F08B9407B4BB
:100B700009EF06F007B009EF06F01EC620F61FC603
:100B800021F61CC61EF61DC61FF61AC61CF61BC68D
:100B90001DF606C608F607C609F604C606F605C61B
:100BA00007F602C604F603C605F626C628F627C6CB
:100BB00029F624C626F625C627F622C624F623C61D
:100BC00025F60EC610F60FC611F60CC60EF60DC6AB
:100BD0000FF60AC60CF60BC60DF62EC630F62FC65B
:100BE00031F62CC62EF62DC62FF62AC62CF62BC6AD
:100BF0002DF616C618F617C619F614C616F615C63B
:100C000017F612C614F613C615F613EC37F0C1EC3E
:100C100036F0077C07AC24EF06F0C274C2B41EEFB6
:100C200006F0C3CFB7F5C4CFB8F50501D890B833F7
:100C3000B733D890B833B73325EF06F0C3CF55F1AB
:100C4000C4CF56F125EF06F0C28207B492EF06F04A
:100C500047C14BF148C14CF149C14DF14AC14EF178
:100C60005EC162F15FC163F160C164F161C165F1B0
:100C700096C1B6F197C1B7F198C1B8F199C1B9F170
:100C80009AC1BAF19BC1BBF19CC1BCF19DC1BDF140
:100C90009EC1BEF19FC1BFF1A0C1C0F1A1C1C1F110
:100CA000A2C1C2F1A3C1C3F1A4C1C4F1A5C1C5F1E0
:100CB000A6C1C6F1A7C1C7F1A8C1C8F1A9C1C9F1B0
:100CC000AAC1CAF1ABC1CBF1ACC1CCF1ADC1CDF180
:100CD000AEC1CEF1AFC1CFF1B0C1D0F1B1C1D1F150
:100CE000B2C1D2F1B3C1D3F1B4C1D4F1B5C1D5F120
:100CF000B7C5B9F5B8C5BAF5B9C5BBF5BAC5BCF540
:100D0000010155515B2756515C23E86A5D230E2E85
:100D100092EF06F05CC157F15DC158F15B6B5C6B03
:100D20005D6B078E0201002FA0EF0BF03C0E006FF1
:100D30001950E00BE00AE866128817BE02D017B41B
:100D4000108E00C10CF101C10DF102C10EF103C101
:100D50000FF104C110F105C111F106C112F107C173
:100D600013F108C114F109C115F10AC116F10BC143
:100D700017F134C135F105012F51000AD8B46CEFD9
:100D800007F005012F51010AD8B4F6EF06F005016E
:100D90002F51020AD8B437EF07F005012F51030A8B
:100DA000D8B437EF07F005012F51040AD8B437EF54
:100DB00007F005012F51050AD8B437EF07F00501F8
:100DC0002F51060AD8B437EF07F005012F51070A53
:100DD000D8B437EF07F005012F51320AD8B4F4EF39
:100DE00006F02F6B6CEF07F06CEF07F0050157670B
:100DF00001EF07F0586701EF07F0596701EF07F0BF
:100E00005A6705EF07F06CEF07F05BC500F15CC5B2
:100E100001F15DC502F15EC503F10101010E046F30
:100E2000000E056F000E066F000E076F32EC35F0F6
:100E300000C15BF501C15CF502C15DF503C15EF562
:100E400000672AEF07F001672AEF07F002672AEF31
:100E500007F003676CEF07F057C55BF558C55CF505
:100E600059C55DF55AC55EF50F886CEF07F00501B1
:100E700030673DEF07F06CEF07F00FBE52EF07F061
:100E800010A057EF07F0010147674EEF07F04867E2
:100E90004EEF07F049674EEF07F04A6752EF07F051
:100EA00057EF07F007AE57EF07F069EF07F00501BE
:100EB000312F6CEF07F03C0E316F302F6CEF07F0E5
:100EC0000101000E626FE00E636FA50E646F010EEC
:100ED000656F0501306B0F880501666B37B772EFE0
:100EE00007F066810CC100F10DC101F10EC102F1E4
:100EF0000FC103F110C104F111C105F112C106F1D6
:100F000013C107F114C108F115C109F116C10AF1A5
:100F100017C10BF135C134F100C10CF101C10DF164
:100F200002C10EF103C10FF104C110F105C111F1AD
:100F300006C112F107C113F108C114F109C115F17D
:100F40000AC116F10BC117F134C135F101018A67ED
:100F5000B1EF07F08B67B1EF07F08C67B1EF07F0E7
:100F60008D67B5EF07F0E5EF07F08EC100F18FC197
:100F700001F190C102F191C103F10101010E046F71
:100F8000000E056F000E066F000E076F32EC35F095
:100F900000C18EF101C18FF102C190F103C191F145
:100FA0000067DAEF07F00167DAEF07F00267DAEFC0
:100FB00007F00367E5EF07F08AC18EF18BC18FF16F
:100FC0008CC190F18DC191F10F80D57ED5BE6DD0D1
:100FD000D6CF47F1D7CF48F145C149F1E86AE8CF0C
:100FE0004AF118BE02D018A0108C109047C100F131
:100FF00048C101F149C102F14AC103F101010A0EE0
:10100000046F000E056F000E066F000E076F32ECC6
:1010100035F003AF1080010154A71BEF08F00F9AC1
:101020000F9C0F9E0101000E5E6F600E5F6F3D0E04
:10103000606F080E616F010147BF2BEF08F0486732
:101040002BEF08F049672BEF08F04A672BEF08F009
:10105000F28850EF08F0F2985E6B5F6B606B616B2B
:10106000966B976B986B996B9A6B9B6B9C6B9D6B5C
:101070009E6B9F6BA06BA16BA26BA36BA46BA56B0C
:10108000A66BA76BA86BA96BAA6BAB6BAC6BAD6BBC
:10109000AE6BAF6BB06BB16BB26BB36BB46BB56B6C
:1010A000D76AD66A0101456B466B0CC100F10DC1D0
:1010B00001F10EC102F10FC103F110C104F111C120
:1010C00005F112C106F113C107F114C108F115C1F0
:1010D00009F116C10AF117C10BF135C134F1A0EFC6
:1010E0000BF0A0EF0BF00201002FB7EF0AF0D59E36
:1010F000D6CF47F1D7CF48F145C149F1E86AE8CFEB
:101100004AF1D76AD66A0101456B466BD58E1950F4
:10111000E00BE00AE866128817BE02D017B4108E02
:1011200016AE1B8C00C10CF101C10DF102C10EF114
:1011300003C10FF104C110F105C111F106C112F193
:1011400007C113F108C114F109C115F10AC116F163
:101150000BC117F134C135F10FA0109A11B8BCEFD3
:1011600008F00101620E046F010E056F000E066F9C
:10117000000E076FC5EF08F00101A70E046F020E05
:10118000056F000E066F000E076F47C100F148C1E2
:1011900001F149C102F14AC103F132EC35F003BF5C
:1011A000D8EF08F018BE02D018A0108C11B00F8034
:1011B0000CC100F10DC101F10EC102F10FC103F12B
:1011C00010C104F111C105F112C106F113C107F1FB
:1011D00014C108F115C109F116C10AF117C10BF1CB
:1011E00035C134F102013C0E006F00C10CF101C1A8
:1011F0000DF102C10EF103C10FF104C110F105C1DF
:1012000011F106C112F107C113F108C114F109C1AE
:1012100015F10AC116F10BC117F134C135F1050101
:101220002F51000AD8B4C0EF09F005012F51010A6F
:10123000D8B44AEF09F005012F51020AD8B48BEF58
:1012400009F005012F51030AD8B48BEF09F005010D
:101250002F51040AD8B48BEF09F005012F51050A6C
:10126000D8B48BEF09F005012F51060AD8B48BEFE3
:1012700009F005012F51070AD8B48BEF09F00501D9
:101280002F51320AD8B448EF09F02F6BC0EF09F0A4
:10129000C0EF09F00501576755EF09F0586755EFA2
:1012A00009F0596755EF09F05A6759EF09F0C0EF97
:1012B00009F05BC500F15CC501F15DC502F15EC5D9
:1012C00003F10101010E046F000E056F000E066FA1
:1012D000000E076F32EC35F000C15BF501C15CF523
:1012E00002C15DF503C15EF500677EEF09F001679D
:1012F0007EEF09F002677EEF09F00367C0EF09F0A7
:1013000057C55BF558C55CF559C55DF55AC55EF521
:101310000F88C0EF09F00501306791EF09F0C0EFC9
:1013200009F00FBEA6EF09F010A0ABEF09F0010124
:101330004767A2EF09F04867A2EF09F04967A2EFFB
:1013400009F04A67A6EF09F0ABEF09F007AEABEF83
:1013500009F0BDEF09F00501312FC0EF09F03C0E97
:10136000316F302FC0EF09F00101000E626FE00E07
:10137000636FA50E646F010E656F0501306B0F88FA
:101380000501666B37B7C6EF09F066810CC100F145
:101390000DC101F10EC102F10FC103F110C104F141
:1013A00011C105F112C106F113C107F114C108F111
:1013B00015C109F116C10AF117C10BF135C134F19C
:1013C00000C10CF101C10DF102C10EF103C10FF119
:1013D00004C110F105C111F106C112F107C113F1E9
:1013E00008C114F109C115F10AC116F10BC117F1B9
:1013F00034C135F101018A6705EF0AF08B6705EF0B
:101400000AF08C6705EF0AF08D6709EF0AF039EFF3
:101410000AF08EC100F18FC101F190C102F191C1BA
:1014200003F10101010E046F000E056F000E066F3F
:10143000000E076F32EC35F000C18EF101C18FF163
:1014400002C190F103C191F100672EEF0AF001672C
:101450002EEF0AF002672EEF0AF0036739EF0AF069
:101460008AC18EF18BC18FF18CC190F18DC191F148
:101470000F80109047C100F148C101F149C102F14C
:101480004AC103F101010A0E046F000E056F000E40
:10149000066F000E076F32EC35F003AF10800101CC
:1014A00054A75FEF0AF00F9A0F9C0F9E0101000EE8
:1014B0005E6F600E5F6F3D0E606F080E616F47C11B
:1014C00000F148C101F149C102F14AC103F1010132
:1014D000140E046F050E056F000E066F000E076FE9
:1014E00032EC35F003AF78EF0AF0F2889DEF0AF0A6
:1014F000F2985E6B5F6B606B616B966B976B986B32
:10150000996B9A6B9B6B9C6B9D6B9E6B9F6BA06B9F
:10151000A16BA26BA36BA46BA56BA66BA76BA86B4F
:10152000A96BAA6BAB6BAC6BAD6BAE6BAF6BB06BFF
:10153000B16BB26BB36BB46BB56B0CC100F10DC189
:1015400001F10EC102F10FC103F110C104F111C18B
:1015500005F112C106F113C107F114C108F115C15B
:1015600009F116C10AF117C10BF135C134F10400BC
:101570008BB4C2EF0AF010ACC2EF0AF08B84109C5F
:10158000C3EF0AF08B9407B415EF0BF007B015EF1B
:101590000BF01EC620F61FC621F61CC61EF61DC681
:1015A0001FF61AC61CF61BC61DF606C608F607C6A9
:1015B00009F604C606F605C607F602C604F603C613
:1015C00005F626C628F627C629F624C626F625C619
:1015D00027F622C624F623C625F60EC610F60FC639
:1015E00011F60CC60EF60DC60FF60AC60CF60BC6A3
:1015F0000DF62EC630F62FC631F62CC62EF62DC6A9
:101600002FF62AC62CF62BC62DF616C618F617C6C8
:1016100019F614C616F615C617F612C614F613C632
:1016200015F613EC37F0C1EC36F0077C07AC30EF61
:101630000BF0C274C2B42AEF0BF0C3CFB7F5C4CF1E
:10164000B8F50501D890B833B733D890B833B7336D
:1016500031EF0BF0C3CF55F1C4CF56F131EF0BF0A2
:10166000C28207B49EEF0BF047C14BF148C14CF169
:1016700049C14DF14AC14EF15EC162F15FC163F1F2
:1016800060C164F161C165F196C1B6F197C1B7F16E
:1016900098C1B8F199C1B9F19AC1BAF19BC1BBF136
:1016A0009CC1BCF19DC1BDF19EC1BEF19FC1BFF106
:1016B000A0C1C0F1A1C1C1F1A2C1C2F1A3C1C3F1D6
:1016C000A4C1C4F1A5C1C5F1A6C1C6F1A7C1C7F1A6
:1016D000A8C1C8F1A9C1C9F1AAC1CAF1ABC1CBF176
:1016E000ACC1CCF1ADC1CDF1AEC1CEF1AFC1CFF146
:1016F000B0C1D0F1B1C1D1F1B2C1D2F1B3C1D3F116
:10170000B4C1D4F1B5C1D5F1B7C5B9F5B8C5BAF50D
:10171000B9C5BBF5BAC5BCF5010155515B2756519A
:101720005C23E86A5D230E2E9EEF0BF05CC157F13F
:101730005DC158F15B6B5C6B5D6B078EA0EF0BF0CE
:1017400002C0E0FF005001C0D8FF1000A6B2A6EF13
:101750000BF00CC0A9FF0BC0A8FFA69EA69CA684F8
:10176000F29E550EA76EAA0EA76EA682F28EA694C2
:10177000A6B2B8EF0BF00C2A1200A96EA69EA69C8A
:10178000A680A8500C2A120004012C0E826F38EC9F
:101790000FF02DEC36F00C50BDEC0BF0E8CF00F163
:1017A0000C50BDEC0BF0E8CF01F101AFDDEF0BF019
:1017B0000101FF0E026FFF0E036FD0EC35F02967B9
:1017C000E9EF0BF00401200E826F38EC0FF0EEEF22
:1017D0000BF004012D0E826F38EC0FF0FAEC33F0B1
:1017E0001200076A0F6A106A116A126A0F010D0E61
:1017F000C16E860EC06E030EC26E0F01680E896E3A
:10180000130E926E080E8A6E8A6AF30E936E8B6ABE
:10181000900E946EC80EBDEC0BF0E8CFE8FF109868
:10182000E8A0108810A805D00E0E216E8E0E226E34
:1018300004D00F0E216E8F0E226ECBEC37F0F18E9E
:10184000F19EFC0EBDEC0BF0E8CF0BF00BA011806D
:101850000BA211820BA411840BA81188C90EBDEC38
:101860000BF0E8CF16F0CA0EBDEC0BF0E8CF17F086
:10187000CB0EBDEC0BF0E8CF18F0CC0EBDEC0BF0AE
:10188000E8CF19F01B6A1C6A0E6A01015B6B5C6B86
:101890005D6B576B586BF29A0101476B486B496B54
:1018A0004A6B4B6B4C6B4D6B4E6B4F6B506B516B74
:1018B000526B456B466BD76AD66A0F01280ED56E00
:1018C000F28A9D90B00ECD6E01015E6B5F6B606B16
:1018D000616B626B636B646B656B666B676B686B8C
:1018E000696B536B546BCF6ACE6A0F9A0F9C0F9E35
:1018F0009D80760ECA6E9D8202013C0E006FCC6AFE
:10190000160EBDEC0BF0E8CF00F1170EBDEC0BF09E
:10191000E8CF01F1180EBDEC0BF0E8CF02F1190E83
:10192000BDEC0BF0E8CF03F1010103AFB2EF0CF017
:101930002DEC36F0160E0C6E00C10BF0A6EC0BF081
:10194000170E0C6E01C10BF0A6EC0BF0180E0C6E0E
:1019500002C10BF0A6EC0BF0190E0C6E03C10BF0DC
:10196000A6EC0BF000C18AF101C18BF102C18CF130
:1019700003C18DF100C18EF101C18FF102C190F15F
:1019800003C191F11A0EBDEC0BF0E8CF00F11B0E74
:10199000BDEC0BF0E8CF01F11C0EBDEC0BF0E8CF75
:1019A00002F11D0EBDEC0BF0E8CF03F1010103AF16
:1019B00008EF0DF02DEC36F01A0E0C6E00C10BF096
:1019C000A6EC0BF01B0E0C6E01C10BF0A6EC0BF09D
:1019D0001C0E0C6E02C10BF0A6EC0BF01D0E0C6E73
:1019E00003C10BF0A6EC0BF01A0EBDEC0BF0E8CF28
:1019F00000F11B0EBDEC0BF0E8CF01F11C0EBDECAD
:101A00000BF0E8CF02F11D0EBDEC0BF0E8CF03F1B7
:101A100000C192F101C193F102C194F103C195F1AA
:101A2000240EAC6E900EAB6E240EAC6E080EB86E2B
:101A3000000EB06E1F0EAF6E0401806B816B0F0144
:101A4000900EAB6E0F019D8A0301806B816BC26BA0
:101A50008B9253EC3CF053EC3CF0880EBDEC0BF059
:101A6000E8CF00F1890EBDEC0BF0E8CF01F10101E8
:101A700001AF53EF0DF02DEC36F0880E0C6E00C167
:101A80000BF0A6EC0BF0890E0C6E01C10BF0A6EC6E
:101A90000BF0880EBDEC0BF0E8CF00F1890EBDEC29
:101AA0000BF0E8CF01F100C140F601C141F602C1DF
:101AB00042F603C143F6ABEC3FF032EC3AF0200EB5
:101AC000BDEC0BF0E8CF2FF505012F51FF0AD8A48C
:101AD00071EF0DF02F6B200E0C6E2FC50BF0A6ECE6
:101AE0000BF00501010E306F3C0E316F250EBDEC81
:101AF0000BF0E8CF00F1260EBDEC0BF0E8CF01F1C2
:101B0000270EBDEC0BF0E8CF02F1280EBDEC0BF078
:101B1000E8CF03F1010103AFA8EF0DF02DEC36F093
:101B2000250E0C6E00C10BF0A6EC0BF0260E0C6E11
:101B300001C10BF0A6EC0BF0270E0C6E02C10BF0EE
:101B4000A6EC0BF0280E0C6E03C10BF0A6EC0BF00C
:101B500000C157F501C158F502C159F503C15AF545
:101B600000C15BF501C15CF502C15DF503C15EF525
:101B7000290EBDEC0BF0E8CF5FF5050160515F5D0C
:101B8000D8A05FC560F505012F51020A0EE181B8AA
:101B9000D5EF0DF00501602FD2EF0DF05FC560F5B8
:101BA000D5EF0DF081BAEAEF3FF0210EBDEC0BF05E
:101BB000E8CF00F1220EBDEC0BF0E8CF01F1230ECF
:101BC000BDEC0BF0E8CF02F1240EBDEC0BF0E8CF3A
:101BD00003F1010103AF1BEF0EF02DEC36F0210EE7
:101BE0000C6E00C10BF0A6EC0BF0220E0C6E01C1C6
:101BF0000BF0A6EC0BF0230E0C6E02C10BF0A6EC62
:101C00000BF0240E0C6E03C10BF0A6EC0BF0210EB2
:101C1000BDEC0BF0E8CF00F1220EBDEC0BF0E8CFED
:101C200001F1230EBDEC0BF0E8CF02F1240EBDEC68
:101C30000BF0E8CF03F100C161F501C162F502C10B
:101C400063F503C164F57AEC39F07CEC38F0D4EC40
:101C500037F005012F51030A12E005012F51040A44
:101C60001DE005012F51050A24E005012F51060A48
:101C700032E005012F51070A38E07EEF0EF0B0C5C3
:101C800000F101010F0E001701010051000A36E0BA
:101C900001010051050A32E07BEF0EF0B0C500F102
:101CA00001010F0E001701010051000A27E07BEF30
:101CB0000EF00501B051000A21E00501B051150AEE
:101CC0001DE00501B051300A19E00501B051450A87
:101CD00015E07BEF0EF00501B051000A0FE00501A1
:101CE000B051300A0BE07BEF0EF00501B051000A55
:101CF00005E07BEF0EF081BAEAEF3FF065EC37F0DC
:101D000007900001F28EF28C12BE20EF1FF007B098
:101D10008FEF31F00FB02BEF2BF010BE2BEF2BF02D
:101D200012B82BEF2BF00FB8C8EF24F0030180514D
:101D300081197F0BD8B48FEF31F013EE00F0815191
:101D40007F0BE126812BE7CFE8FFE00BD8B48FEFC4
:101D500031F023EE82F0C2513F0BD926E7CFDFFFEF
:101D6000C22BDF50780AD8A48FEF31F007808EC1E4
:101D700000F18FC101F190C102F191C103F10101A4
:101D8000040E046F000E056F000E066F000E076F45
:101D900032EC35F000AFD6EF0EF00101030E8E6F7E
:101DA000000E8F6F000E906F000E916F0301825135
:101DB000720AD8B410EF2BF08251520AD8B410EF47
:101DC0002BF08251750AD8B410EF2BF08251630AC0
:101DD000D8B449EF2EF08251690AD8B4BFEF27F08A
:101DE00082517A0AD8B4D2EF28F08251490AD8B485
:101DF0005EEF27F08251500AD8B47CEF26F0825172
:101E0000700AD8B4BFEF26F08251540AD8B4EAEF72
:101E100026F08251740AD8B430EF27F08251410A7B
:101E2000D8B44CEF0FF082516D0AD8B456EF13F0CE
:101E300082514D0AD8B46FEF13F08251730AD8B4AF
:101E400040EF2AF08251530AD8B4A5EF2AF082510C
:101E50004C0AD8B4D2EF1AF08251760AD8B4FEEF09
:101E600013F08251590AD8B4A7EF12F080EF2EF088
:101E7000040114EE00F080517F0BE12682C4E7FFDD
:101E8000802B120004010D0E826F38EC0FF00A0E49
:101E9000826F38EC0FF012000401410E826F38ECB3
:101EA0000FF003018351310AD8B4C7EF11F00301D9
:101EB0008351320AD8B4F7EF10F003018351330A8B
:101EC000D8B480EF10F003018351340AD8B470EF16
:101ED0000FF004013F0E826F38EC0FF07EEF2EF012
:101EE000CC0EBDEC0BF0E8CF0BF004012C0E826F92
:101EF00038EC0FF003018451310AD8B494EF0FF09D
:101F000003018451300AD8B496EF0FF003018451D5
:101F10004D0AD8B4A0EF0FF003018451540AD8B48D
:101F2000A7EF0FF0BEEF0FF08A8401D08A940BAEBA
:101F300004D00BAC02D00BBA21D0E00E0B1218D09B
:101F40001F0E0B168539E844E00B0B1211D0E00E82
:101F50000B166EEC36F085C332F186C333F1010106
:101F6000296B7BEC36F0F2EC35F000511F0B0B12B5
:101F7000CC0E0C6E0BC00BF0A6EC0BF00401340E73
:101F8000826F38EC0FF004012C0E826F38EC0FF0EA
:101F9000CC0EBDEC0BF0E8CF19F08AB406D00401EA
:101FA000300E826F38EC0FF005D00401310E826FD5
:101FB00038EC0FF004012C0E826F38EC0FF019385A
:101FC000E840070BE8CF82F40401300E822738EC9A
:101FD0000FF004012C0E826F38EC0FF02DEC36F070
:101FE00019501F0BE8CF00F1D0EC35F032C182F46C
:101FF0000401300E822738EC0FF033C182F4040163
:10200000300E822738EC0FF004012C0E826F38EC72
:102010000FF02DEC36F02CC000F100AF0BD0FF0E0E
:10202000016FFF0E026FFF0E036F04012D0E826F12
:1020300038EC0FF0D0EC35F031C182F40401300EF1
:10204000822738EC0FF032C182F40401300E82276F
:1020500038EC0FF033C182F40401300E822738ECE3
:102060000FF004012C0E826F38EC0FF02DEC36F0DF
:102070002BC000F1D0EC35F031C182F40401300EF8
:10208000822738EC0FF032C182F40401300E82272F
:1020900038EC0FF033C182F40401300E822738ECA3
:1020A0000FF004012C0E826F38EC0FF02DEC36F09F
:1020B0002DC000F100AF0BD0FF0E016FFF0E026FBD
:1020C000FF0E036F04012D0E826F38EC0FF0D0EC81
:1020D00035F031C182F40401300E822738EC0FF064
:1020E00032C182F40401300E822738EC0FF033C184
:1020F00082F40401300E822738EC0FF07EEF2EF0D0
:10210000CB0EBDEC0BF0E8CF0BF004012C0E826F70
:1021100038EC0FF003018451450AD8B4A4EF10F055
:1021200003018451440AD8B4A7EF10F0030184518D
:10213000300AD8B4AAEF10F003018451310AD8B4A0
:10214000AEEF10F0B9EF10F00B9EB3EF10F00B8E66
:10215000B3EF10F0FC0E0B16B3EF10F0FC0E0B16E5
:102160000B80B3EF10F0CB0E0C6E0BC00BF0A6EC97
:102170000BF00401330E826F38EC0FF004012C0ECB
:10218000826F38EC0FF0CB0EBDEC0BF0E8CF18F0FF
:1021900018BED2EF10F00401450E826F38EC0FF03C
:1021A000D7EF10F00401440E826F38EC0FF00401F9
:1021B0002C0E826F38EC0FF00401300E826F38EC79
:1021C0000FF004012C0E826F38EC0FF018B0F0EF16
:1021D00010F00401300E826F38EC0FF0F5EF10F0C4
:1021E0000401310E826F38EC0FF07EEF2EF0CA0E34
:1021F000BDEC0BF0E8CF0BF004012C0E826F38EC35
:102200000FF003018451450AD8B433EF11F00301F4
:102210008451440AD8B436EF11F0030184514D0AB9
:10222000D8B43FEF11F003018451410AD8B439EF1B
:1022300011F003018451460AD8B43CEF11F00301B8
:102240008451560AD8B447EF11F003018451500A63
:10225000D8B452EF11F003018451520AD8B455EFAB
:1022600011F05EEF11F00B9E58EF11F00B8E58EF4E
:1022700011F00B9C58EF11F00B8C58EF11F0FC0E85
:102280000B1685C3E8FF030B0B1258EF11F0C70EB6
:102290000B1685C3E8FF070BE846E846E8460B1235
:1022A00058EF11F00B8458EF11F00B9458EF11F028
:1022B000CA0E0C6E0BC00BF0A6EC0BF0CA0EBDECF8
:1022C0000BF0E8CF17F00401320E826F38EC0FF0FC
:1022D00004012C0E826F38EC0FF017BE77EF11F06F
:1022E0000401450E826F38EC0FF07CEF11F0040111
:1022F000440E826F38EC0FF004012C0E826F38EC24
:102300000FF017C0E8FF030BE8CF82F40401300E92
:10231000822738EC0FF004012C0E826F38EC0FF09E
:1023200017BC9AEF11F00401410E826F38EC0FF0E8
:102330009FEF11F00401460E826F38EC0FF004019C
:102340002C0E826F38EC0FF017C0E8FF380BE84214
:10235000E842E842E8CF82F40401300E822738ECEC
:102360000FF004012C0E826F38EC0FF017B4C0EFA1
:1023700011F00401520E826F38EC0FF0C5EF11F02E
:102380000401500E826F38EC0FF07EEF2EF0C90E74
:10239000BDEC0BF0E8CF0BF004012C0E826F38EC93
:1023A0000FF003018451450AD8B4E5EF11F00301A1
:1023B0008451440AD8B4E8EF11F0030184514D0A66
:1023C000D8B4EBEF11F0F9EF11F00B9EF3EF11F031
:1023D0000B8EF3EF11F0F80E0B1685C3E8FF070B19
:1023E0000B12F3EF11F0C90E0C6E0BC00BF0A6EC44
:1023F0000BF00401310E826F38EC0FF004012C0E4B
:10240000826F38EC0FF0C90EBDEC0BF0E8CF16F080
:1024100016BE06D00401450E826F38EC0FF005D0D1
:102420000401440E826F38EC0FF004012C0E826F11
:1024300038EC0FF016C0E8FF070BE8CF82F4040178
:10244000300E822738EC0FF004012C0E826F38EC2E
:102450000FF007802DEC36F027C0E8FF003B00436B
:102460000043030BD0EC35F033C182F40401300E8D
:10247000822738EC0FF004012C0E826F38EC0FF03D
:102480002DEC36F027C001F1019F019D28C000F11D
:102490000101D0EC35F02FC182F40401300E822707
:1024A00038EC0FF030C182F40401300E822738EC92
:1024B0000FF031C182F40401300E822738EC0FF0A6
:1024C00032C182F40401300E822738EC0FF033C1A0
:1024D00082F40401300E822738EC0FF004012C0E38
:1024E000826F38EC0FF02DEC36F029C001F12AC0D4
:1024F00000F1D89001330033D8900133003301014B
:10250000D0EC35F02FC182F40401300E822738EC74
:102510000FF030C182F40401300E822738EC0FF046
:1025200031C182F40401300E822738EC0FF032C141
:1025300082F40401300E822738EC0FF033C182F4AC
:102540000401300E822738EC0FF07EEF2EF0FC0EE7
:10255000BDEC0BF0E8CF0BF003018351520AD8B465
:10256000DEEF12F003018351720AD8B4E1EF12F0EA
:1025700003018351500AD8B4E4EF12F003018351F0
:10258000700AD8B4E7EF12F003018351550AD8B4AA
:10259000EAEF12F003018351750AD8B4EDEF12F09F
:1025A00003018351430AD8B4F6EF12F003018351BB
:1025B000630AD8B4F9EF12F002EF13F00B90FCEFBE
:1025C00012F00B80FCEF12F00B92FCEF12F00B827A
:1025D000FCEF12F00B94FCEF12F00B84FCEF12F006
:1025E0000B96FCEF12F00B86FCEF12F00B98FCEF51
:1025F00012F00B88FCEF12F0FC0E0C6E0BC00BF00F
:10260000A6EC0BF00401590E826F38EC0FF011901C
:10261000119211941198FC0EBDEC0BF0E8CF0BF069
:102620000BA011800BA211820BA411840BA811889E
:1026300011A022EF13F00401520E826F38EC0FF05C
:1026400027EF13F00401720E826F38EC0FF011A81F
:1026500031EF13F00401430E826F38EC0FF036EFC8
:1026600013F00401630E826F38EC0FF011A240EFFB
:1026700013F00401500E826F38EC0FF045EF13F0A9
:102680000401700E826F38EC0FF011A44FEF13F0BD
:102690000401550E826F38EC0FF054EF13F0040173
:1026A000750E826F38EC0FF07EEF2EF004016D0E88
:1026B000826F38EC0FF003018351300AD8B4AEEFCB
:1026C00013F003018351310AD8B4C1EF13F00301B1
:1026D0008351320AD8B4D4EF13F080EF2EF0040106
:1026E0004D0E826F38EC0FF06EEC36F084C331F192
:1026F00085C332F186C333F10101296B7BEC36F0DF
:10270000F2EC35F003018351300AD8B496EF13F0A0
:1027100003018351310AD8B49EEF13F003018351B2
:10272000320AD8B4A6EF13F080EF2EF0FD0E0C6E37
:1027300000C10BF0A6EC0BF0AEEF13F0FE0E0C6E2A
:1027400000C10BF0A6EC0BF0C1EF13F0FF0E0C6E06
:1027500000C10BF0A6EC0BF0D4EF13F00401300E27
:10276000826F38EC0FF004012C0E826F38EC0FF002
:102770002DEC36F0FD0EBDEC0BF0E8CF00F1E5EFEF
:1027800013F00401310E826F38EC0FF004012C0EAF
:10279000826F38EC0FF02DEC36F0FE0EBDEC0BF036
:1027A000E8CF00F1E5EF13F00401320E826F38EC50
:1027B0000FF02DEC36F004012C0E826F38EC0FF088
:1027C000FF0EBDEC0BF0E8CF00F1D0EC35F031C1DD
:1027D00082F40401300E822738EC0FF032C182F40B
:1027E0000401300E822738EC0FF033C182F404016B
:1027F000300E822738EC0FF07EEF2EF0030183516C
:10280000300AD8B4A3EF15F003018351310AD8B4CC
:10281000DAEF15F003018351320AD8B48FEF17F0C5
:1028200003018351330AD8B444EF19F003018351F3
:10283000340AD8B4EAEF19F003018351730AD8B40B
:1028400085EF14F003018351760AD8B487EF14F0B2
:1028500003018351740AD8B472EF14F00301835159
:10286000540AD8B437EF14F0D8A480EF2EF0040146
:10287000760E826F38EC0FF00401540E826F38EC44
:102880000FF007840001880E0C6E6EEC36F0298183
:10289000030184512D0AD8B450EF14F0010129919D
:1028A00085C32FF186C330F187C331F188C332F17C
:1028B00089C333F17BEC36F0F2EC35F000C10BF05C
:1028C000A6EC0BF001C10BF0A6EC0BF0880EBDECF2
:1028D0000BF0E8CF40F6890EBDEC0BF0E8CF41F6E7
:1028E0007DEF14F00401760E826F38EC0FF00401D6
:1028F000740E826F38EC0FF007840001880E0C6EA6
:10290000C4EC0BF0079429EF25F085EC14F00401DA
:10291000760E826F38EC0FF00401760E826F38EC81
:102920000FF00784AAEC32F004012C0E826F38EC11
:102930000FF00101036B026B3BC601F13AC600F1D7
:1029400001AFA8EF14F00101FF0E026FFF0E036F3D
:10295000D0EC35F02967AFEF14F0B4EF14F00401B8
:102960002D0E826F38EC0FF02FC182F40401300E6F
:10297000822738EC0FF030C182F40401300E822738
:1029800038EC0FF031C182F40401300E822738ECAC
:102990000FF032C182F40401300E822738EC0FF0C0
:1029A00033C182F40401300E822738EC0FF00401A9
:1029B0002C0E826F38EC0FF00101036B026B3DC6E9
:1029C00001F13CC600F101AFEBEF14F00101FF0E85
:1029D000026FFF0E036FD0EC35F02967F2EF14F0B1
:1029E000F7EF14F004012D0E826F38EC0FF02FC1B9
:1029F00082F40401300E822738EC0FF030C182F4EB
:102A00000401300E822738EC0FF031C182F404014A
:102A1000300E822738EC0FF032C182F40401300E00
:102A2000822738EC0FF033C182F40401300E822784
:102A300038EC0FF004012C0E826F38EC0FF001011E
:102A4000036B026B3FC601F13EC600F101AF2EEFF2
:102A500015F00101FF0E026FFF0E036FD0EC35F091
:102A6000296735EF15F03AEF15F004012D0E826F4E
:102A700038EC0FF02FC182F40401300E822738ECBD
:102A80000FF030C182F40401300E822738EC0FF0D1
:102A900031C182F40401300E822738EC0FF032C1CC
:102AA00082F40401300E822738EC0FF033C182F437
:102AB0000401300E822738EC0FF004012C0E826FD7
:102AC00038EC0FF00101036B026B37C601F136C61B
:102AD00000F101AF71EF15F00101FF0E026FFF0E63
:102AE000036FD0EC35F0296778EF15F07DEF15F026
:102AF00004012D0E826F38EC0FF02FC182F4040117
:102B0000300E822738EC0FF030C182F40401300E11
:102B1000822738EC0FF031C182F40401300E822795
:102B200038EC0FF032C182F40401300E822738EC09
:102B30000FF033C182F40401300E822738EC0FF01D
:102B4000079429EF25F00401760E826F38EC0FF020
:102B50000401300E826F38EC0FF004012C0E826FEE
:102B600038EC0FF09BEC36F02DEC36F000C600F19F
:102B700001C601F1D0EC35F030C182F40401300E11
:102B8000822738EC0FF031C182F40401300E822725
:102B900038EC0FF032C182F40401300E822738EC99
:102BA0000FF033C182F40401300E822738EC0FF0AD
:102BB00029EF25F00401760E826F38EC0FF0040146
:102BC000310E826F38EC0FF007840101036B026B4A
:102BD00002C600F103C601F101AFF3EF15F0FF0EDD
:102BE000026FFF0E036F0101076B066B04C604F151
:102BF00005C605F105AF01EF16F0FF0E066FFF0EDB
:102C0000076F37EC35F00101076B066B06C604F160
:102C100007C605F105AF11EF16F0FF0E066FFF0EA8
:102C2000076F37EC35F00101076B066B08C604F13E
:102C300009C605F105AF21EF16F0FF0E066FFF0E76
:102C4000076F37EC35F0D8900101033302330133BD
:102C50000033D89001010333023301330033040100
:102C60002C0E826F38EC0FF00101036B026B01C177
:102C700001F100C100F101AF43EF16F00101FF0EB9
:102C8000026FFF0E036FD0EC35F029674AEF16F0A4
:102C90004FEF16F004012D0E826F38EC0FF02FC1AC
:102CA00082F40401300E822738EC0FF030C182F438
:102CB0000401300E822738EC0FF031C182F4040198
:102CC000300E822738EC0FF032C182F40401300E4E
:102CD000822738EC0FF033C182F40401300E8227D2
:102CE00038EC0FF00101036B026B0AC600F10BC652
:102CF00001F101AF80EF16F0FF0E026FFF0E036FC0
:102D00000101076B066B0CC604F10DC605F105AF9A
:102D10008EEF16F0FF0E066FFF0E076F37EC35F0E3
:102D20000101076B066B0EC604F10FC605F105AF76
:102D30009EEF16F0FF0E066FFF0E076F37EC35F0B3
:102D40000101076B066B10C604F111C605F105AF52
:102D5000AEEF16F0FF0E066FFF0E076F37EC35F083
:102D6000D89001010333023301330033D8900101BD
:102D7000033302330133003304012C0E826F38EC2D
:102D80000FF00101036B026B01C101F100C100F101
:102D900001AFD0EF16F00101FF0E026FFF0E036FBF
:102DA000D0EC35F02967D7EF16F0DCEF16F0040110
:102DB0002D0E826F38EC0FF02FC182F40401300E1B
:102DC000822738EC0FF030C182F40401300E8227E4
:102DD00038EC0FF031C182F40401300E822738EC58
:102DE0000FF032C182F40401300E822738EC0FF06C
:102DF00033C182F40401300E822738EC0FF0010158
:102E0000036B026B12C600F113C601F101AF0DEFA7
:102E100017F0FF0E026FFF0E036F0101076B066BC9
:102E200014C604F115C605F105AF1BEF17F0FF0E30
:102E3000066FFF0E076F37EC35F00101076B066B6D
:102E400016C604F117C605F105AF2BEF17F0FF0EFC
:102E5000066FFF0E076F37EC35F00101076B066B4D
:102E600018C604F119C605F105AF3BEF17F0FF0EC8
:102E7000066FFF0E076F37EC35F0D8900101033372
:102E8000023301330033D89001010333023301339D
:102E9000003304012C0E826F38EC0FF00101036B3C
:102EA000026B01C101F100C100F101AF5DEF17F04C
:102EB0000101FF0E026FFF0E036FD0EC35F02967A2
:102EC00064EF17F069EF17F004012D0E826F38ECF4
:102ED0000FF02FC182F40401300E822738EC0FF07E
:102EE00030C182F40401300E822738EC0FF031C17A
:102EF00082F40401300E822738EC0FF032C182F4E4
:102F00000401300E822738EC0FF033C182F4040143
:102F1000300E822738EC0FF0079429EF25F00401DA
:102F2000760E826F38EC0FF00401320E826F38ECAF
:102F30000FF007840101036B026B1AC600F11BC678
:102F400001F101AFA8EF17F0FF0E026FFF0E036F44
:102F50000101076B066B1CC604F11DC605F105AF28
:102F6000B6EF17F0FF0E066FFF0E076F37EC35F068
:102F70000101076B066B1EC604F11FC605F105AF04
:102F8000C6EF17F0FF0E066FFF0E076F37EC35F038
:102F90000101076B066B20C604F121C605F105AFE0
:102FA000D6EF17F0FF0E066FFF0E076F37EC35F008
:102FB000D89001010333023301330033D89001016B
:102FC000033302330133003304012C0E826F38ECDB
:102FD0000FF00101036B026B01C101F100C100F1AF
:102FE00001AFF8EF17F00101FF0E026FFF0E036F44
:102FF000D0EC35F02967FFEF17F004EF18F004016B
:103000002D0E826F38EC0FF02FC182F40401300EC8
:10301000822738EC0FF030C182F40401300E822791
:1030200038EC0FF031C182F40401300E822738EC05
:103030000FF032C182F40401300E822738EC0FF019
:1030400033C182F40401300E822738EC0FF0010105
:10305000036B026B22C600F123C601F101AF35EF0D
:1030600018F0FF0E026FFF0E036F0101076B066B76
:1030700024C604F125C605F105AF43EF18F0FF0E95
:10308000066FFF0E076F37EC35F00101076B066B1B
:1030900026C604F127C605F105AF53EF18F0FF0E61
:1030A000066FFF0E076F37EC35F00101076B066BFB
:1030B00028C604F129C605F105AF63EF18F0FF0E2D
:1030C000066FFF0E076F37EC35F0D8900101033320
:1030D000023301330033D89001010333023301334B
:1030E000003304012C0E826F38EC0FF00101036BEA
:1030F000026B01C101F100C100F101AF85EF18F0D1
:103100000101FF0E026FFF0E036FD0EC35F029674F
:103110008CEF18F091EF18F004012D0E826F38EC4F
:103120000FF02FC182F40401300E822738EC0FF02B
:1031300030C182F40401300E822738EC0FF031C127
:1031400082F40401300E822738EC0FF032C182F491
:103150000401300E822738EC0FF033C182F40401F1
:10316000300E822738EC0FF00101036B026B2AC688
:1031700000F12BC601F101AFC2EF18F0FF0E026F94
:10318000FF0E036F0101076B066B2CC604F12DC601
:1031900005F105AFD0EF18F0FF0E066FFF0E076FB9
:1031A00037EC35F00101076B066B2EC604F12FC614
:1031B00005F105AFE0EF18F0FF0E066FFF0E076F89
:1031C00037EC35F00101076B066B30C604F131C6F0
:1031D00005F105AFF0EF18F0FF0E066FFF0E076F59
:1031E00037EC35F0D890010103330233013300335B
:1031F000D8900101033302330133003304012C0E54
:10320000826F38EC0FF00101036B026B01C101F119
:1032100000C100F101AF12EF19F00101FF0E026FC2
:10322000FF0E036FD0EC35F0296719EF19F01EEF90
:1032300019F004012D0E826F38EC0FF02FC182F4CB
:103240000401300E822738EC0FF030C182F4040103
:10325000300E822738EC0FF031C182F40401300EB9
:10326000822738EC0FF032C182F40401300E82273D
:1032700038EC0FF033C182F40401300E822738ECB1
:103280000FF0079429EF25F00401760E826F38ECD9
:103290000FF00401330E826F38EC0FF004012C0E96
:1032A000826F38EC0FF085C382F438EC0FF0640EB7
:1032B0000D6E03018551320A02E16A0E0D6E0301A3
:1032C0008551330A02E1700E0D6E03018551340AF7
:1032D00002E1760E0D6E03018551350A02E17C0E86
:1032E0000D6E03018551360A02E1820E0D6E030157
:1032F0008651780A65E00DC00CF06EEC36F029813D
:10330000030187512D0AD8B488EF19F001012991E2
:1033100088C32FF189C330F18AC331F18BC332F1F5
:103320008CC333F17BEC36F0F2EC35F000C10BF0DE
:10333000A6EC0BF001C10BF0A6EC0BF06EEC36F036
:10334000298103018E512D0AD8B4A9EF19F001018A
:1033500029918FC32FF190C330F191C331F192C302
:1033600032F193C333F17BEC36F0F2EC35F000C16F
:103370000BF0A6EC0BF001C10BF0A6EC0BF06EEC21
:1033800036F02981030195512D0AD8B4CAEF19F0FE
:103390000101299196C32FF197C330F198C331F100
:1033A00099C332F19AC333F17BEC36F0F2EC35F08D
:1033B00000C10BF0A6EC0BF001C10BF0A6EC0BF07A
:1033C0000DC00CF0C4EC0BF0C4EC0BF0C4EC0BF033
:1033D00029EF25F00401760E826F38EC0FF004011E
:1033E000340E826F38EC0FF003018451780AD8B4A0
:1033F000C2EF1AF03E0E0C6E6EEC36F0298103011E
:1034000085512D0AD8B407EF1AF00101299186C31E
:103410002FF187C330F188C331F189C332F18AC3F8
:1034200033F17BEC36F0F2EC35F000C10BF0A6EC9A
:103430000BF001C10BF0A6EC0BF06EEC36F029811D
:1034400003018C512D0AD8B428EF1AF001012991FB
:103450008DC32FF18EC330F18FC331F190C332F1A0
:1034600091C333F17BEC36F0F2EC35F000C10BF098
:10347000A6EC0BF001C10BF0A6EC0BF06EEC36F0F5
:103480002981030193512D0AD8B449EF1AF00101A3
:10349000299194C32FF195C330F196C331F197C3AD
:1034A00032F198C333F17BEC36F0F2EC35F000C129
:1034B0000BF0A6EC0BF001C10BF0A6EC0BF06EECE0
:1034C00036F0298103019A512D0AD8B46AEF1AF017
:1034D000010129919BC32FF19CC330F19DC331F1B0
:1034E0009EC332F19FC333F17BEC36F0F2EC35F042
:1034F00000C10BF0A6EC0BF001C10BF0A6EC0BF039
:103500006EEC36F029810301A1512D0AD8B48BEF5E
:103510001AF001012991A2C32FF1A3C330F1A4C372
:1035200031F1A5C332F1A6C333F17BEC36F0F2ECF6
:1035300035F000C10BF0A6EC0BF001C10BF0A6ECCE
:103540000BF06EEC36F029810301A8512D0AD8B496
:10355000ACEF1AF001012991A9C32FF1AAC330F1F0
:10356000ABC331F1ACC332F1ADC333F17BEC36F018
:10357000F2EC35F000C10BF0A6EC0BF001C10BF042
:10358000A6EC0BF03E0E0C6EC4EC0BF0C4EC0BF092
:10359000C4EC0BF0C4EC0BF0C4EC0BF0C4EC0BF07F
:1035A00029EF25F003018351300AD8B4CCEF1FF086
:1035B00003018351310AD8B4F9EF20F0030183519C
:1035C000320AD8B467EF21F003018351330AD8B42B
:1035D00077EF21F003018351340AD8B487EF21F04B
:1035E00003018351350AD8B4CDEF24F00301835190
:1035F000360AD8B4FBEF24F003018351370AD8B45C
:10360000A5EF1DF003018351380AD8B443EF1EF033
:1036100003018351460AD8B421EF24F003018351FA
:103620004D0AD8B41EEF1CF0030183516D0AD8B4C3
:1036300038EF1CF0030183515A0AD8B473EF20F01D
:1036400003018351490AD8B4FBEF25F003018351EC
:10365000500AD8B42DEF25F003018351540AD8B491
:10366000A6EF25F003018351630AD8B458EF1CF08C
:1036700003018351430AD8B450EF1DF00301835175
:10368000730AD8B456EF1CF003018351610AD8B411
:103690006BEF1BF003018351650AD8B41CEF20F0D7
:1036A00003018351450AD8B42AEF20F00301835166
:1036B000620AD8B438EF20F003018351420AD8B42B
:1036C00046EF20F003018351760AD8B454EF20F07E
:1036D000D8A480EF2EF004014C0E826F38EC0FF06E
:1036E0000401610E826F38EC0FF07CEC38F00401BD
:1036F0002C0E826F38EC0FF02DEC36F0AFC500F1D8
:103700000101D0EC35F031C182F40401300E822782
:1037100038EC0FF032C182F40401300E822738EC0D
:103720000FF033C182F40401300E822738EC0FF021
:1037300004012C0E826F38EC0FF02DEC36F0B0C582
:1037400000F10101D0EC35F031C182F40401300EFA
:10375000822738EC0FF032C182F40401300E822748
:1037600038EC0FF033C182F40401300E822738ECBC
:103770000FF004012C0E826F38EC0FF02DEC36F0B8
:10378000B1C500F10101D0EC35F031C182F4040182
:10379000300E822738EC0FF032C182F40401300E73
:1037A000822738EC0FF033C182F40401300E8227F7
:1037B00038EC0FF004012C0E826F38EC0FF02DEC7A
:1037C00036F0B2C500F10101D0EC35F031C182F420
:1037D0000401300E822738EC0FF032C182F404016C
:1037E000300E822738EC0FF033C182F40401300E22
:1037F000822738EC0FF004012C0E826F38EC0FF0AA
:103800002DEC36F0B6C500F10101D0EC35F031C138
:1038100082F40401300E822738EC0FF032C182F4BA
:103820000401300E822738EC0FF033C182F404011A
:10383000300E822738EC0FF029EF25F06EEC36F0D1
:1038400084C333F17BEC36F0F2EC35F0200E0C6ED5
:1038500000C10BF0A6EC0BF000C12FF505012F51B4
:10386000000A06E005012F51010A02E016EC39F0CA
:1038700004014C0E826F38EC0FF004014D0E826F84
:1038800038EC0FF004012C0E826F38EC0FF02DECA9
:1038900036F02FC500F1D0EC35F033C182F40401CD
:1038A000300E822738EC0FF029EF25F0EAEF3FF0D9
:1038B00004014C0E826F38EC0FF00401630E826F2E
:1038C00038EC0FF0D4EC37F004012C0E826F38EC9A
:1038D0000FF06DEC1CF029EF25F02DEC36F0B5C59E
:1038E00000F10101003B0F0E0017D0EC35F033C1A1
:1038F00082F40401300E822738EC0FF0B5C500F1D8
:1039000001010F0E01010017D0EC35F033C182F434
:103910000401300E822738EC0FF004012D0E826F67
:1039200038EC0FF0B4C500F10101003B0F0E001799
:10393000D0EC35F033C182F40401300E822738EC2C
:103940000FF0B4C500F101010F0E01010017D0EC1A
:1039500035F033C182F40401300E822738EC0FF0C9
:1039600004012D0E826F38EC0FF0B3C500F1010198
:10397000003B0F0E0017D0EC35F033C182F4040188
:10398000300E822738EC0FF0B3C500F101010F0EA5
:1039900001010017D0EC35F033C182F40401300E80
:1039A000822738EC0FF00401200E826F38EC0FF004
:1039B000B2C500F10F0E01010017D0EC35F033C194
:1039C00082F40401300E822738EC0FF00401200E3F
:1039D000826F38EC0FF0B1C500F101010101003B2D
:1039E0000F0E0017D0EC35F033C182F40401300E15
:1039F000822738EC0FF0B1C500F101010F0E010173
:103A00000017D0EC35F033C182F40401300E822768
:103A100038EC0FF004013A0E826F38EC0FF0B0C5AD
:103A200000F10101003B0F0E0017D0EC35F033C15F
:103A300082F40401300E822738EC0FF0B0C500F19B
:103A400001010F0E01010017D0EC35F033C182F4F3
:103A50000401300E822738EC0FF004013A0E826F19
:103A600038EC0FF0AFC500F10101003B0F0E00175D
:103A7000D0EC35F033C182F40401300E822738ECEB
:103A80000FF0AFC500F101010F0E0017D0EC35F0BB
:103A900033C182F40401300E822738EC0FF012009B
:103AA00084C3E8FF0F0BE83AE8CFB5F585C3E8FF1C
:103AB0000F0B0501B51387C3E8FF0F0BE83AE8CFFA
:103AC000B4F588C3E8FF0F0B0501B4138AC3E8FF00
:103AD0000F0BE83AE8CFB3F58BC3E8FF0F0B0501F6
:103AE000B3138DC3E8FF0F0BE8CFB2F58FC3E8FF28
:103AF0000F0BE83AE8CFB1F590C3E8FF0F0B0501D3
:103B0000B11392C3E8FF0F0BE83AE8CFB0F593C3C7
:103B1000E8FF0F0B0501B01395C3E8FF0F0BE83A60
:103B2000E8CFAFF596C3E8FF0F0B0501AF132FECFD
:103B300038F004014C0E826F38EC0FF00401430E94
:103B4000826F38EC0FF062EF1CF0078404014C0E1A
:103B5000826F38EC0FF00401370E826F38EC0FF0F3
:103B600004012C0E826F38EC0FF005012E51130A60
:103B700006E005012E51170A0DE040EF1EF001018D
:103B8000000E006F000E016F100E026F000E036F2B
:103B9000D3EF1DF00101000E006F000E016F000E4B
:103BA000026F010E036FD0EC35F02AC182F40401DC
:103BB000300E822738EC0FF02BC182F40401300E56
:103BC000822738EC0FF02CC182F40401300E8227DA
:103BD00038EC0FF02DC182F40401300E822738EC4E
:103BE0000FF02EC182F40401300E822738EC0FF062
:103BF0002FC182F40401300E822738EC0FF030C15F
:103C000082F40401300E822738EC0FF031C182F4C7
:103C10000401300E822738EC0FF032C182F4040127
:103C2000300E822738EC0FF033C182F40401300EDD
:103C3000822738EC0FF004012C0E826F38EC0FF065
:103C40000101200E006F000E016F000E026F000ECA
:103C5000036FD0EC35F031C182F40401300E8227BD
:103C600038EC0FF032C182F40401300E822738ECB8
:103C70000FF033C182F40401300E822738EC0FF0CC
:103C8000079429EF25F00501216B226B236B246B30
:103C900004014C0E826F38EC0FF00401380E826F75
:103CA00038EC0FF004012C0E826F38EC0FF001019C
:103CB000200E006F000E016F000E026F000E036FEA
:103CC000D0EC35F02AC182F40401300E822738ECA2
:103CD0000FF02BC182F40401300E822738EC0FF074
:103CE0002CC182F40401300E822738EC0FF02DC174
:103CF00082F40401300E822738EC0FF02EC182F4DA
:103D00000401300E822738EC0FF02FC182F4040139
:103D1000300E822738EC0FF030C182F40401300EEF
:103D2000822738EC0FF031C182F40401300E822773
:103D300038EC0FF032C182F40401300E822738ECE7
:103D40000FF033C182F40401300E822738EC0FF0FB
:103D500004012C0E826F38EC0FF025C500F126C54A
:103D600001F127C502F128C503F10101200E046FFE
:103D7000000E056F000E066F000E076F63EC35F046
:103D800000C133F501C134F502C135F503C136F583
:103D9000D0EC35F02AC182F40401300E822738ECD1
:103DA0000FF02BC182F40401300E822738EC0FF0A3
:103DB0002CC182F40401300E822738EC0FF02DC1A3
:103DC00082F40401300E822738EC0FF02EC182F409
:103DD0000401300E822738EC0FF02FC182F4040169
:103DE000300E822738EC0FF030C182F40401300E1F
:103DF000822738EC0FF031C182F40401300E8227A3
:103E000038EC0FF032C182F40401300E822738EC16
:103E10000FF033C182F40401300E822738EC0FF02A
:103E200042EC0FF0050133671DEF1FF034671DEF03
:103E30001FF035671DEF1FF0366702D0BBEF1FF094
:103E4000129E21C500F122C501F123C502F124C54E
:103E500003F1899A400EC76E200EC66E9E96C69ECE
:103E60000B0EC96EFF0E9EB602D0E82EFCD79E96B2
:103E7000C69E02C1C9FFFF0E9EB602D0E82EFCD737
:103E80009E96C69E01C1C9FFFF0E9EB602D0E82EC7
:103E9000FCD79E96C69E00C1C9FFFF0E9EB602D0FB
:103EA000E82EFCD79E96C69EC952FF0E9EB602D043
:103EB000E82EFCD70501200E326F040114EE00F04D
:103EC00080517F0BE1269E96C69EC952FF0E9EB67C
:103ED00002D0E82EFCD7C9CFE7FF0401802B0501F3
:103EE000322F5DEF1FF0898A33C500F134C501F12F
:103EF00035C502F136C503F10101010E046F000E54
:103F0000056F000E066F000E076F32EC35F000C132
:103F100033F501C134F502C135F503C136F50501AC
:103F200033679AEF1FF034679AEF1FF035679AEF07
:103F30001FF0366702D0BBEF1FF021C500F122C58C
:103F400001F123C502F124C503F10101200E046F24
:103F5000000E056F000E066F000E076F37EC35F090
:103F600000C121F501C122F502C123F503C124F5E9
:103F7000128E80EF2EF00401450E826F38EC0FF0A8
:103F800004014F0E826F38EC0FF00401460E826F71
:103F900038EC0FF029EF25F00784ABEC3FF02DEC67
:103FA00036F02DC500F1D0EC35F004014C0E826FD7
:103FB00038EC0FF00401300E826F38EC0FF0040182
:103FC0002C0E826F38EC0FF031C182F40401300EF8
:103FD000822738EC0FF032C182F40401300E8227C0
:103FE00038EC0FF033C182F40401300E822738EC34
:103FF0000FF004012C0E826F38EC0FF02DEC36F030
:104000002EC500F1D0EC35F031C182F40401300E40
:10401000822738EC0FF032C182F40401300E82277F
:1040200038EC0FF033C182F40401300E822738ECF3
:104030000FF0079429EF25F004014C0E826F38EC45
:104040000FF00401650E826F38EC0FF0D6EC39F0FA
:1040500029EF25F004014C0E826F38EC0FF00401BB
:10406000450E826F38EC0FF0EDEC39F029EF25F0BA
:1040700004014C0E826F38EC0FF00401620E826F67
:1040800038EC0FF01BEC3AF029EF25F004014C0E50
:10409000826F38EC0FF00401420E826F38EC0FF0A3
:1040A00004EC3AF029EF25F004014C0E826F38EC55
:1040B0000FF00401760E826F38EC0FF004012C0E25
:1040C000826F38EC0FF010A807D00401310E826F18
:1040D00038EC0FF029EF25F00401300E826F38EC38
:1040E0000FF029EF25F004014C0E826F38EC0FF031
:1040F00004015A0E826F38EC0FF004012C0E826F0F
:1041000038EC0FF0ABEC3FF02DEC36F005012E5102
:10411000130A06E005012E51170A0DE0A4EF20F066
:104120000101000E006F000E016F100E026F000EF5
:10413000036FA4EF20F00101000E006F000E016F6D
:10414000000E026F010E036F0101200E046F000EBE
:10415000056F000E066F000E076F63EC35F0D0ECB4
:1041600035F02AC182F40401300E822738EC0FF0BA
:104170002BC182F40401300E822738EC0FF02CC1E1
:1041800082F40401300E822738EC0FF02DC182F446
:104190000401300E822738EC0FF02EC182F40401A6
:1041A000300E822738EC0FF02FC182F40401300E5C
:1041B000822738EC0FF030C182F40401300E8227E0
:1041C00038EC0FF031C182F40401300E822738EC54
:1041D0000FF032C182F40401300E822738EC0FF068
:1041E00033C182F40401300E822738EC0FF029EF3E
:1041F00025F0078404014C0E826F38EC0FF00401A7
:10420000310E826F38EC0FF004012C0E826F38EC07
:104210000FF025C500F126C501F127C502F128C51B
:1042200003F10101200E046F000E056F000E066FF2
:10423000000E076F63EC35F0D0EC35F02AC182F444
:104240000401300E822738EC0FF02BC182F40401F8
:10425000300E822738EC0FF02CC182F40401300EAE
:10426000822738EC0FF02DC182F40401300E822732
:1042700038EC0FF02EC182F40401300E822738ECA6
:104280000FF02FC182F40401300E822738EC0FF0BA
:1042900030C182F40401300E822738EC0FF031C1B6
:1042A00082F40401300E822738EC0FF032C182F420
:1042B0000401300E822738EC0FF033C182F4040180
:1042C000300E822738EC0FF0079429EF25F0078491
:1042D00004014C0E826F38EC0FF00401320E826F35
:1042E00038EC0FF009EC3CF0079429EF25F0078437
:1042F00004014C0E826F38EC0FF00401330E826F14
:1043000038EC0FF066EC3CF0079404EF21F00784E2
:1043100004014C0E826F38EC0FF00401340E826FF2
:1043200038EC0FF004012C0E826F38EC0FF06EECBD
:1043300036F084C32AF185C32BF186C32CF187C3E1
:104340002DF188C32EF189C32FF18AC330F18BC3BD
:1043500031F18CC332F18DC333F10101296B7BEC58
:1043600036F0F2EC35F0200E046F000E056F000EF3
:10437000066F000E076F43EC35F000C121F501C157
:1043800022F502C123F503C124F55EEC3FF038C5E8
:10439000AFF539C5B0F53AC5B1F53BC5B2F53CC589
:1043A000B3F53DC5B4F53EC5B5F56DEC1CF00401A3
:1043B0002C0E826F38EC0FF03FC500F140C501F1C3
:1043C00041C502F142C503F10101000E046F000E68
:1043D000056F010E066F000E076F63EC35F0D0EC31
:1043E00035F02967F6EF21F0FBEF21F004012D0EE7
:1043F000826F38EC0FF030C182F40401300E822756
:1044000038EC0FF031C182F40401300E822738EC11
:104410000FF004012E0E826F38EC0FF032C182F4DF
:104420000401300E822738EC0FF033C182F404010E
:10443000300E822738EC0FF004012C0E826F38EC1E
:104440000FF02DEC36F043C500F144C501F1AAECA4
:104450002FF004012C0E826F38EC0FF02DEC36F0AB
:1044600045C500F1D0EC35F031C182F40401300EC5
:10447000822738EC0FF032C182F40401300E82271B
:1044800038EC0FF033C182F40401300E822738EC8F
:104490000FF004012C0E826F38EC0FF00101036B5A
:1044A000026B4CC501F14BC500F101AF5DEF22F08D
:1044B0000101FF0E026FFF0E036FD0EC35F029678C
:1044C00064EF22F069EF22F004012D0E826F38ECC8
:1044D0000FF02FC182F40401300E822738EC0FF068
:1044E00030C182F40401300E822738EC0FF031C164
:1044F00082F40401300E822738EC0FF032C182F4CE
:104500000401300E822738EC0FF033C182F404012D
:10451000300E822738EC0FF004012C0E826F38EC3D
:104520000FF00101036B026B4EC501F14DC500F1A7
:1045300001AFA0EF22F00101FF0E026FFF0E036F2B
:10454000D0EC35F02967A7EF22F0ACEF22F00401A0
:104550002D0E826F38EC0FF02FC182F40401300E63
:10456000822738EC0FF030C182F40401300E82272C
:1045700038EC0FF031C182F40401300E822738ECA0
:104580000FF032C182F40401300E822738EC0FF0B4
:1045900033C182F40401300E822738EC0FF004019D
:1045A0002C0E826F38EC0FF00101036B026B50C5CB
:1045B00001F14FC500F101AFE3EF22F00101FF0E61
:1045C000026FFF0E036FD0EC35F02967EAEF22F09F
:1045D000EFEF22F004012D0E826F38EC0FF02FC1A7
:1045E00082F40401300E822738EC0FF030C182F4DF
:1045F0000401300E822738EC0FF031C182F404013F
:10460000300E822738EC0FF032C182F40401300EF4
:10461000822738EC0FF033C182F40401300E822778
:1046200038EC0FF004012C0E826F38EC0FF0010112
:10463000036B026B52C501F151C500F101AF26EFCA
:1046400023F00101FF0E026FFF0E036FD0EC35F077
:1046500029672DEF23F032EF23F004012D0E826F36
:1046600038EC0FF02FC182F40401300E822738ECB1
:104670000FF030C182F40401300E822738EC0FF0C5
:1046800031C182F40401300E822738EC0FF032C1C0
:1046900082F40401300E822738EC0FF033C182F42B
:1046A0000401300E822738EC0FF004012C0E826FCB
:1046B00038EC0FF00101036B026B54C501F153C5D7
:1046C00000F101AF69EF23F00101FF0E026FFF0E51
:1046D000036FD0EC35F0296770EF23F075EF23F00E
:1046E00004012D0E826F38EC0FF02FC182F404010B
:1046F000300E822738EC0FF030C182F40401300E06
:10470000822738EC0FF031C182F40401300E822789
:1047100038EC0FF032C182F40401300E822738ECFD
:104720000FF033C182F40401300E822738EC0FF011
:1047300004012C0E826F38EC0FF00101036B026B49
:1047400056C501F155C500F101AFACEF23F00101F1
:10475000FF0E026FFF0E036FD0EC35F02967B3EF49
:1047600023F0B8EF23F004012D0E826F38EC0FF028
:104770002FC182F40401300E822738EC0FF030C1D3
:1047800082F40401300E822738EC0FF031C182F43C
:104790000401300E822738EC0FF032C182F404019C
:1047A000300E822738EC0FF033C182F40401300E52
:1047B000822738EC0FF004012C0E826F38EC0FF0DA
:1047C0000101036B026B4AC501F149C500F101AF5C
:1047D000EFEF23F00101FF0E026FFF0E036FD0EC2D
:1047E00035F02967F6EF23F0FBEF23F004012D0EDF
:1047F000826F38EC0FF02FC182F40401300E822753
:1048000038EC0FF030C182F40401300E822738EC0E
:104810000FF031C182F40401300E822738EC0FF022
:1048200032C182F40401300E822738EC0FF033C11C
:1048300082F40401300E822738EC0FF0079429EF40
:1048400025F06EEC36F085C32AF186C32BF187C3C1
:104850002CF188C32DF189C32EF18AC32FF18BC3AC
:1048600030F18CC331F18DC332F18EC333F10101CC
:10487000296B7BEC36F0F2EC35F00101010E046F90
:10488000000E056F000E066F000E076F32EC35F05C
:10489000100E046F000E056F000E066F000E076FFE
:1048A00043EC35F000C129F501C12AF502C12BF511
:1048B00003C12CF590EC3BF004014C0E826F38ECF8
:1048C0000FF00401460E826F38EC0FF004012C0E3D
:1048D000826F38EC0FF025C500F126C501F127C520
:1048E00002F128C503F10101100E046F000E056FDF
:1048F000000E066F000E076F63EC35F0D0EC35F05C
:104900002AC182F40401300E822738EC0FF02BC14B
:1049100082F40401300E822738EC0FF02CC182F4AF
:104920000401300E822738EC0FF02DC182F404010F
:10493000300E822738EC0FF02EC182F40401300EC5
:10494000822738EC0FF02FC182F40401300E822749
:1049500038EC0FF030C182F40401300E822738ECBD
:104960000FF031C182F40401300E822738EC0FF0D1
:1049700032C182F40401300E822738EC0FF033C1CB
:1049800082F40401300E822738EC0FF029EF25F075
:104990000F9866EC3CF080EF2EF004014C0E826F15
:1049A00038EC0FF00401350E826F38EC0FF0040183
:1049B0002C0E826F38EC0FF02DEC36F00784B9C561
:1049C00000F10794D0EC35F031C182F40401300ECF
:1049D000822738EC0FF032C182F40401300E8227B6
:1049E00038EC0FF033C182F40401300E822738EC2A
:1049F0000FF029EF25F029EC3CF02DEC36F037C50F
:104A000000F1D0EC35F004014C0E826F38EC0FF061
:104A10000401360E826F38EC0FF004012C0E826F09
:104A200038EC0FF031C182F40401300E822738ECEB
:104A30000FF032C182F40401300E822738EC0FF0FF
:104A400033C182F40401300E822738EC0FF029EFD5
:104A500025F042EC0FF080EF2EF004014C0E826F37
:104A600038EC0FF00401500E826F38EC0FF00401A7
:104A70002C0E826F38EC0FF085C32AF186C32BF120
:104A800087C32CF188C32DF189C32EF18AC32FF17E
:104A90008BC330F18CC331F18DC332F18EC333F14E
:104AA00001017BEC36F0F2EC35F003018451530A3E
:104AB0000DE0030184514D0A38E00401780E826F45
:104AC00038EC0FF042EC0FF080EF2EF00401530EA3
:104AD000826F38EC0FF0250E0C6E00C10BF0A6ECC7
:104AE0000BF0260E0C6E01C10BF0A6EC0BF0270E9E
:104AF0000C6E02C10BF0A6EC0BF0280E0C6E03C17D
:104B00000BF0A6EC0BF000C157F501C158F502C13E
:104B100059F503C15AF500C15BF501C15CF502C14D
:104B20005DF503C15EF50AEF26F004014D0E826FBC
:104B300038EC0FF0290E0C6E00C10BF0A6EC0BF058
:104B400000C15FF500C160F50AEF26F004014C0ECC
:104B5000826F38EC0FF00401540E826F38EC0FF0C6
:104B600004012C0E826F38EC0FF084C32AF185C348
:104B70002BF186C32CF187C32DF188C32EF189C395
:104B80002FF18AC330F18BC331F18DC332F18EC363
:104B900033F101017BEC36F0F2EC35F00101000E4F
:104BA000046F000E056F010E066F000E076F43ECD9
:104BB00035F0210E0C6E00C10BF0A6EC0BF0220EAE
:104BC0000C6E01C10BF0A6EC0BF0230E0C6E02C1B3
:104BD0000BF0A6EC0BF0240E0C6E03C10BF0A6EC50
:104BE0000BF000C161F501C162F502C163F503C1BB
:104BF00064F50AEF26F004014C0E826F38EC0FF0DA
:104C00000401490E826F38EC0FF004012C0E826F04
:104C100038EC0FF0250EBDEC0BF0E8CF00F1260EBE
:104C2000BDEC0BF0E8CF01F1270EBDEC0BF0E8CFA7
:104C300002F1280EBDEC0BF0E8CF03F1D0EC35F01B
:104C4000B3EC33F00401730E826F38EC0FF0040103
:104C50002C0E826F38EC0FF02DEC36F0290EBDECE7
:104C60000BF0E8CF00F1D0EC35F0B3EC33F00401F9
:104C7000730E826F38EC0FF004012C0E826F38EC4B
:104C80000FF05BC500F15CC501F15DC502F15EC5C9
:104C900003F1D0EC35F0B3EC33F00401730E826F06
:104CA00038EC0FF004012C0E826F38EC0FF02DEC75
:104CB00036F060C500F1D0EC35F0B3EC33F0040110
:104CC0006D0E826F38EC0FF004012C0E826F38EC01
:104CD0000FF061C500F162C501F163C502F164C561
:104CE00003F19BEC2EF004012C0E826F38EC0FF0D8
:104CF00042EC0FF080EF2EF083C32AF184C32BF136
:104D000085C32CF186C32DF187C32EF188C32FF103
:104D100089C330F18AC331F18BC332F18CC333F1D3
:104D200001017BEC36F0F2EC35F0160E0C6E00C192
:104D30000BF0A6EC0BF0170E0C6E01C10BF0A6ECFD
:104D40000BF0180E0C6E02C10BF0A6EC0BF0190E56
:104D50000C6E03C10BF0A6EC0BF000C18AF101C18F
:104D60008BF102C18CF103C18DF100C18EF101C143
:104D70008FF102C190F103C191F15EEF27F083C37F
:104D80002AF184C32BF185C32CF186C32DF187C38F
:104D90002EF188C32FF189C330F18AC331F18BC35F
:104DA00032F18CC333F101017BEC36F0F2EC35F0DB
:104DB00000C18AF101C18BF102C18CF103C18DF1F7
:104DC00000C18EF101C18FF102C190F103C191F1D7
:104DD0005EEF27F083C32AF184C32BF185C32CF146
:104DE00086C32DF187C32EF188C32FF189C330F11B
:104DF0008AC331F18CC332F18DC333F101017BECF5
:104E000036F0F2EC35F00101000E046F000E056F74
:104E1000010E066F000E076F43EC35F01A0E0C6E94
:104E200000C10BF0A6EC0BF01B0E0C6E01C10BF0D9
:104E3000A6EC0BF01C0E0C6E02C10BF0A6EC0BF0F6
:104E40001D0E0C6E03C10BF0A6EC0BF000C192F12D
:104E500001C193F102C194F103C195F15EEF27F016
:104E600083C32AF184C32BF185C32CF186C32DF1B2
:104E700087C32EF188C32FF189C330F18AC331F182
:104E80008CC332F18DC333F101017BEC36F0F2ECCF
:104E900035F00101000E046F000E056F010E066F64
:104EA000000E076F43EC35F000C192F101C193F1A0
:104EB00002C194F103C195F15EEF27F0160EBDEC2F
:104EC0000BF0E8CF00F1170EBDEC0BF0E8CF01F1CD
:104ED000180EBDEC0BF0E8CF02F1190EBDEC0BF093
:104EE000E8CF03F1D0EC35F0B3EC33F00401730EEE
:104EF000826F38EC0FF004012C0E826F38EC0FF04B
:104F00008AC100F18BC101F18CC102F18DC103F1A5
:104F1000D0EC35F0B3EC33F00401730E826F38EC53
:104F20000FF004012C0E826F38EC0FF01A0EBDEC5E
:104F30000BF0E8CF00F11B0EBDEC0BF0E8CF01F158
:104F40001C0EBDEC0BF0E8CF02F11D0EBDEC0BF01A
:104F5000E8CF03F19BEC2EF004012C0E826F38ECAD
:104F60000FF092C100F193C101F194C102F195C11A
:104F700003F19BEC2EF042EC0FF080EF2EF00401D9
:104F8000690E826F38EC0FF004012C0E826F38EC42
:104F90000FF00101040E006F000E016F000E026F92
:104FA000000E036FD0EC35F02CC182F40401300EFA
:104FB000822738EC0FF02DC182F40401300E8227D5
:104FC00038EC0FF02EC182F40401300E822738EC49
:104FD0000FF02FC182F40401300E822738EC0FF05D
:104FE00030C182F40401300E822738EC0FF031C159
:104FF00082F40401300E822738EC0FF032C182F4C3
:105000000401300E822738EC0FF033C182F4040122
:10501000300E822738EC0FF004012C0E826F38EC32
:105020000FF001010B0E006F000E016F000E026FFA
:10503000000E036FD0EC35F02CC182F40401300E69
:10504000822738EC0FF02DC182F40401300E822744
:1050500038EC0FF02EC182F40401300E822738ECB8
:105060000FF02FC182F40401300E822738EC0FF0CC
:1050700030C182F40401300E822738EC0FF031C1C8
:1050800082F40401300E822738EC0FF032C182F432
:105090000401300E822738EC0FF033C182F4040192
:1050A000300E822738EC0FF004012C0E826F38ECA2
:1050B0000FF001012D0E006F000E016F000E026F48
:1050C000000E036FD0EC35F02CC182F40401300ED9
:1050D000822738EC0FF02DC182F40401300E8227B4
:1050E00038EC0FF02EC182F40401300E822738EC28
:1050F0000FF02FC182F40401300E822738EC0FF03C
:1051000030C182F40401300E822738EC0FF031C137
:1051100082F40401300E822738EC0FF032C182F4A1
:105120000401300E822738EC0FF033C182F4040101
:10513000300E822738EC0FF004012C0E826F38EC11
:105140000FF0200EF86EF76AF66A04010900F5CF39
:1051500082F438EC0FF00900F5CF82F438EC0FF050
:105160000900F5CF82F438EC0FF00900F5CF82F496
:1051700038EC0FF00900F5CF82F438EC0FF009009D
:10518000F5CF82F438EC0FF00900F5CF82F438EC5B
:105190000FF00900F5CF82F438EC0FF042EC0FF07D
:1051A00080EF2EF08351630AD8A480EF2EF0845153
:1051B000610AD8A480EF2EF085516C0AD8A480EF44
:1051C0002EF08651410A3FE08651440A1BE0865189
:1051D000420AD8B436EF29F08651350AD8B40AEF1E
:1051E00030F08651360AD8B45FEF30F08651370A76
:1051F000D8B4C8EF30F08651380AD8B426EF31F071
:1052000080EF2EF00798079A04017A0E826F38EC2F
:105210000FF00401780E826F38EC0FF00401640E79
:10522000826F38EC0FF00401550E826F38EC0FF0EE
:105230001FEF29F004014C0E826F38EC0FF042ECA6
:105240000FF080EF2EF00788079A04017A0E826F24
:1052500038EC0FF00401410E826F38EC0FF00401BE
:10526000610E826F38EC0FF013EF29F00798078A70
:1052700004017A0E826F38EC0FF00401420E826F47
:1052800038EC0FF00401610E826F38EC0FF013EF71
:1052900029F00101666754EF29F0676754EF29F0A0
:1052A000686754EF29F0696715D04F675FEF29F001
:1052B00050675FEF29F051675FEF29F052670AD01E
:1052C0000101000E006F000E016F000E026F000E54
:1052D000036F120011B80AD00101620E046F010EB3
:1052E000056F000E066F000E076F09D00101A70EB3
:1052F000046F020E056F000E066F000E076F66C189
:1053000000F167C101F168C102F169C103F132EC3A
:1053100035F003BFFCEF29F0119A119C0101000E3A
:10532000046FA80E056F550E066F020E076F66C15B
:1053300000F167C101F168C102F169C103F166C101
:1053400086F167C187F168C188F169C189F132ECE2
:1053500035F003BF0BD00101000E866FA80E876FDA
:10536000550E886F020E896F118A119C0E0EBDECCE
:105370000BF0E8CF18F10F0EBDEC0BF0E8CF19F1F0
:10538000100EBDEC0BF0E8CF1AF1110EBDEC0BF0D6
:10539000E8CF1BF17BEC34F086C104F187C105F145
:1053A00088C106F189C107F132EC35F007823FEC84
:1053B00034F07BEC34F007923FEC34F086C100F11E
:1053C00087C101F188C102F189C103F107923FEC65
:1053D00034F0CC0E046FE00E056F870E066F050EDD
:1053E000076F32EC35F000C118F101C119F102C1AB
:1053F0001AF103C11BF13BD0119C119A0101800EDF
:10540000006F1A0E016F060E026F000E036F4FC180
:1054100004F150C105F151C106F152C107F132EC5E
:1054200035F003AF05D02DEC36F0118C119A120037
:105430000E0EBDEC0BF0E8CF18F10F0EBDEC0BF02B
:10544000E8CF19F1100EBDEC0BF0E8CF1AF1110EF8
:10545000BDEC0BF0E8CF1BF14FC100F150C101F1E1
:1054600051C102F152C103F107823FEC34F018C17F
:1054700000F119C101F11AC102F11BC103F11200BF
:105480000401730E826F38EC0FF004012C0E826F52
:1054900038EC0FF0078462C166F163C167F164C143
:1054A00068F165C169F14BC14FF14CC150F14DC17B
:1054B00051F14EC152F157C159F158C15AF10794F7
:1054C00066EC2AF042EC0FF080EF2EF066C100F19E
:1054D00067C101F168C102F169C103F10101D0ECBA
:1054E00035F0B3EC33F00401630E826F38EC0FF04B
:1054F00004012C0E826F38EC0FF04FC100F150C147
:1055000001F151C102F152C103F10101D0EC35F0BA
:10551000B3EC33F00401660E826F38EC0FF0040137
:105520002C0E826F38EC0FF02DEC36F059C100F1E3
:105530005AC101F10101D0EC35F0B3EC33F00401B4
:10554000740E826F38EC0FF0120010820401530EBB
:10555000826F38EC0FF004012C0E826F38EC0FF0E4
:1055600083C32AF184C32BF185C32CF186C32DF1AB
:1055700087C32EF188C32FF189C330F18AC331F17B
:105580008BC332F18CC333F101017BEC36F0F2ECCA
:1055900035F000C166F101C167F102C168F103C1D4
:1055A00069F18EC32AF18FC32BF190C32CF191C303
:1055B0002DF192C32EF193C32FF194C330F195C313
:1055C00031F196C332F197C333F101017BEC36F030
:1055D000F2EC35F000C14FF101C150F102C151F1BF
:1055E00003C152F16EEC36F099C32FF19AC330F13A
:1055F0009BC331F19CC332F19DC333F101017BECBC
:1056000036F0F2EC35F000C159F101C15AF166EC07
:105610002AF004012C0E826F38EC0FF01FEF2BF0F4
:10562000118E18A002D018AE108C17BE02D017A48D
:10563000108E8251520A02E10F8201D00F928251E4
:10564000750A02E1108401D010948251550A02E1DA
:10565000108601D0109611A003D011A401D010849F
:10566000078410B28DEF2BF010A479EF2BF0B6C1A8
:1056700066F1B7C167F1B8C168F1B9C169F1BAC1E2
:105680006AF1BBC16BF1BCC16CF1BDC16DF1BEC1B2
:105690006EF1BFC16FF1C0C170F1C1C171F1C2C182
:1056A00072F1C3C173F1C4C174F1C5C175F1C6C152
:1056B00076F1C7C177F1C8C178F1C9C179F1CAC122
:1056C0007AF1CBC17BF1CCC17CF1CDC17DF1CEC1F2
:1056D0007EF1CFC17FF1D0C180F1D1C181F1D2C1C2
:1056E00082F1D3C183F1D4C184F1D5C185F181EFB9
:1056F0002BF062C166F163C167F164C168F165C1F5
:1057000069F14BC14FF14CC150F14DC151F14EC146
:1057100052F157C159F158C15AF107940FA0AFEF98
:105720002BF0010192679CEF2BF093679CEF2BF01D
:1057300094679CEF2BF09567A0EF2BF0AFEF2BF069
:1057400049EC29F092C104F193C105F194C106F12D
:1057500095C107F132EC35F003BF46EF2EF049EC6E
:1057600029F00101000E046F000E056F010E066F97
:10577000000E076F63EC35F011A02CD011A22AD0D7
:10578000D0EC35F0296701D007D004012D0E826FCF
:1057900038EC0FF044EF2EF030C182F40401300EEB
:1057A000822738EC0FF031C182F40401300E8227D9
:1057B00038EC0FF032C182F40401300E822738EC4D
:1057C0000FF033C182F40401300E822738EC0FF061
:1057D00044EF2EF012A8C5D0129819C01AF01A3A48
:1057E0001A42070E1A1600011A50000AD8B47DEFAB
:1057F0002CF000011A50010AD8B409EF2CF0000176
:105800001A50020AD8B407EF2CF0AFEF2CF0AFEF2C
:105810002CF02DEC36F029C001F12AC000F1D8900F
:1058200001330033D890013300330101630E046F5C
:10583000000E056F000E066F000E076F63EC35F06B
:10584000280E046F000E056F000E066F000E076F26
:1058500032EC35F000C12CF02DEC36F027C001F110
:10586000019F019D28C000F10101A40E046F000EEC
:10587000056F000E066F000E076F63EC35F000C178
:105880002BF000C104F101C105F102C106F103C111
:1058900007F1640E006F000E016F000E026F000E24
:1058A000036F32EC35F0050E046F000E056F000E2D
:1058B000066F000E076F63EC35F000C104F101C103
:1058C00005F102C106F103C107F12DEC36F02CC041
:1058D00000F132EC35F000C12DF02DC0E8FF050FCE
:1058E0002C5C03E78A84AFEF2CF02DC0E8FF0A0F91
:1058F0002C5C01E68A94AFEF2CF000C124F101C1C9
:1059000025F102C126F103C127F12DEC36F033EC6D
:1059100036F019501F0BE8CF00F10101640E046F3F
:10592000000E056F000E066F000E076F43EC35F09A
:1059300024C104F125C105F126C106F127C107F1F3
:1059400032EC35F003BF02D08A9401D08A8424C19E
:1059500000F125C101F126C102F127C103F146EF93
:105960002EF000C124F101C125F102C126F103C1CD
:1059700027F110AE4CD0109E00C108F101C109F111
:1059800002C10AF103C10BF1D0EC35F030C1D6F100
:1059900031C1D7F132C1D8F133C1D9F108C100F119
:1059A00009C101F10AC102F10BC103F101016C0E41
:1059B000046F070E056F000E066F000E076F32ECC6
:1059C00035F003BF04D00101550EDA6F1CD008C1B9
:1059D00000F109C101F10AC102F10BC103F101019A
:1059E000A40E046F060E056F000E066F000E076F03
:1059F00032EC35F003BF04D001017F0EDA6F03D023
:105A00000101FF0EDA6F1B8E11AE46EF2EF024C19E
:105A100000F125C101F126C102F127C103F110A453
:105A200019EF2DF00401750E826F38EC0FF01EEFA8
:105A30002DF00401720E826F38EC0FF004012C0E71
:105A4000826F38EC0FF0D0EC35F029672DEF2DF098
:105A50000401200E826F30EF2DF004012D0E826FB5
:105A600038EC0FF030C182F40401300E822738EC9C
:105A70000FF031C182F40401300E822738EC0FF0B0
:105A800004012E0E826F38EC0FF032C182F4040153
:105A9000300E822738EC0FF033C182F40401300E4F
:105AA000822738EC0FF004016D0E826F38EC0FF096
:105AB00004012C0E826F38EC0FF04FC100F150C181
:105AC00001F151C102F152C103F10101D0EC35F0F5
:105AD000B3EC33F00401480E826F38EC0FF0040190
:105AE0007A0E826F38EC0FF004012C0E826F38ECC6
:105AF0000FF066C100F167C101F168C102F169C12F
:105B000003F10101D0EC35F0B3EC33F00401630E86
:105B1000826F38EC0FF004012C0E826F38EC0FF01E
:105B200066C100F167C101F168C102F169C103F109
:105B300001010A0E046F000E056F000E066F000EC5
:105B4000076F43EC35F0000E046F120E056F000E68
:105B5000066F000E076F63EC35F0D0EC35F02AC10C
:105B600082F40401300E822738EC0FF02BC182F44E
:105B70000401300E822738EC0FF02CC182F40401AE
:105B8000300E822738EC0FF02DC182F40401300E64
:105B9000822738EC0FF02EC182F40401300E8227E8
:105BA00038EC0FF02FC182F40401300E822738EC5C
:105BB0000FF030C182F40401300E822738EC0FF070
:105BC00004012E0E826F38EC0FF031C182F4040113
:105BD000300E822738EC0FF032C182F40401300E0F
:105BE000822738EC0FF033C182F40401300E822793
:105BF00038EC0FF00401730E826F38EC0FF00401E3
:105C00002C0E826F38EC0FF02DEC36F059C100F1FC
:105C10005AC101F1AAEC2FF00FB212EF2EF00FA033
:105C200044EF2EF004012C0E826F38EC0FF0200EA2
:105C3000F86EF76AF66A04010900F5CF82F438ECD1
:105C40000FF00900F5CF82F438EC0FF00900F5CF22
:105C500082F438EC0FF00900F5CF82F438EC0FF045
:105C60000900F5CF82F438EC0FF00900F5CF82F48B
:105C700038EC0FF00900F5CF82F438EC0FF0090092
:105C8000F5CF82F438EC0FF042EC0FF00F9080EF7C
:105C90002EF00401630E826F38EC0FF004012C0E1D
:105CA000826F38EC0FF086EC2EF004012C0E826F20
:105CB00038EC0FF0F9EC2EF004012C0E826F38EC6A
:105CC0000FF075EC2FF004012C0E826F38EC0FF002
:105CD0000101F80E006FCD0E016F660E026F030E0C
:105CE000036F9BEC2EF004012C0E826F38EC0FF04A
:105CF0008BEC2FF042EC0FF080EF2EF042EC0FF027
:105D00000301C26B079010928FEF31F0D8900E0E06
:105D1000BDEC0BF0E8CF00F10F0EBDEC0BF0E8CFBF
:105D200001F1100EBDEC0BF0E8CF02F1110EBDEC4D
:105D30000BF0E8CF03F10101000E046F000E056FB8
:105D4000010E066F000E076F63EC35F0D0EC35F0F6
:105D50002AC182F40401300E822738EC0FF02BC1E7
:105D600082F40401300E822738EC0FF02CC182F44B
:105D70000401300E822738EC0FF02DC182F40401AB
:105D8000300E822738EC0FF02EC182F40401300E61
:105D9000822738EC0FF02FC182F40401300E8227E5
:105DA00038EC0FF030C182F40401300E822738EC59
:105DB0000FF031C182F40401300E822738EC0FF06D
:105DC00004012E0E826F38EC0FF032C182F4040110
:105DD000300E822738EC0FF033C182F40401300E0C
:105DE000822738EC0FF004016D0E826F38EC0FF053
:105DF0001200120EBDEC0BF0E8CF00F1130EBDEC5B
:105E00000BF0E8CF01F1140EBDEC0BF0E8CF02F17E
:105E1000150EBDEC0BF0E8CF03F101010A0E046F83
:105E2000000E056F000E066F000E076F43EC35F095
:105E3000000E046F120E056F000E066F000E076F46
:105E400063EC35F0D0EC35F02AC182F40401300E59
:105E5000822738EC0FF02BC182F40401300E822728
:105E600038EC0FF02CC182F40401300E822738EC9C
:105E70000FF02DC182F40401300E822738EC0FF0B0
:105E80002EC182F40401300E822738EC0FF02FC1AE
:105E900082F40401300E822738EC0FF030C182F416
:105EA0000401300E822738EC0FF004012E0E826FB1
:105EB00038EC0FF031C182F40401300E822738EC47
:105EC0000FF032C182F40401300E822738EC0FF05B
:105ED00033C182F40401300E822738EC0FF0040144
:105EE000730E826F38EC0FF012000A0EBDEC0BF04F
:105EF000E8CF00F10B0EBDEC0BF0E8CF01F10C0E7A
:105F0000BDEC0BF0E8CF02F10D0EBDEC0BF0E8CFCD
:105F100003F1AAEF2FF0060EBDEC0BF0E8CF00F175
:105F2000070EBDEC0BF0E8CF01F1080EBDEC0BF055
:105F3000E8CF02F1090EBDEC0BF0E8CF03F1AAEFB8
:105F40002FF001012DEC36F0078457C100F158C144
:105F500001F107940101E80E046F800E056F000E39
:105F6000066F000E076F43EC35F0000E046F040E51
:105F7000056F000E066F000E076F63EC35F0880E9C
:105F8000046F130E056F000E066F000E076F32ECE4
:105F900035F00A0E046F000E056F000E066F000E3E
:105FA000076F63EC35F0D0EC35F001012967DEEFC7
:105FB0002FF00401200E826FE1EF2FF004012D0E6F
:105FC000826F38EC0FF030C182F40401300E82276A
:105FD00038EC0FF031C182F40401300E822738EC26
:105FE0000FF032C182F40401300E822738EC0FF03A
:105FF00004012E0E826F38EC0FF033C182F40401DD
:10600000300E822738EC0FF00401430E826F38EC1B
:106010000FF0120087C32AF188C32BF189C32CF13A
:106020008AC32DF18BC32EF18CC32FF18DC330F1B8
:106030008EC331F190C332F191C333F10101296B69
:106040007BEC36F0F2EC35F00101000E046F000E2F
:10605000056F010E066F000E076F43EC35F00E0E54
:106060000C6E00C10BF0A6EC0BF00F0E0C6E01C114
:106070000BF0A6EC0BF0100E0C6E02C10BF0A6ECB0
:106080000BF0110E0C6E03C10BF0A6EC0BF004012B
:106090007A0E826F38EC0FF004012C0E826F38EC10
:1060A0000FF00401350E826F38EC0FF004012C0E56
:1060B000826F38EC0FF086EC2EF01FEF29F087C3CB
:1060C0002AF188C32BF189C32CF18AC32DF18BC32C
:1060D0002EF18CC32FF18DC330F18EC331F190C3FB
:1060E00032F191C333F10101296B7BEC36F0F2EC14
:1060F00035F0880E046F130E056F000E066F000E4C
:10610000076F37EC35F0000E046F040E056F000EBC
:10611000066F000E076F43EC35F00101E80E046FC7
:10612000800E056F000E066F000E076F63EC35F0F2
:106130000A0E0C6E00C10BF0A6EC0BF00B0E0C6EF1
:1061400001C10BF0A6EC0BF00C0E0C6E02C10BF0B3
:10615000A6EC0BF00D0E0C6E03C10BF0A6EC0BF0D1
:1061600004017A0E826F38EC0FF004012C0E826F5E
:1061700038EC0FF00401360E826F38EC0FF004019A
:106180002C0E826F38EC0FF075EC2FF01FEF29F01A
:1061900087C32AF188C32BF189C32CF18AC32DF15F
:1061A0008BC32EF18CC32FF18DC330F18FC331F12E
:1061B00090C332F191C333F101017BEC36F0F2EC84
:1061C00035F0000E046F120E056F000E066F000E04
:1061D000076F43EC35F001010A0E046F000E056FE6
:1061E000000E066F000E076F63EC35F0120E0C6E9A
:1061F00000C10BF0A6EC0BF0130E0C6E01C10BF0FE
:10620000A6EC0BF0140E0C6E02C10BF0A6EC0BF01A
:10621000150E0C6E03C10BF0A6EC0BF004017A0E08
:10622000826F38EC0FF004012C0E826F38EC0FF007
:106230000401370E826F38EC0FF004012C0E826FD0
:1062400038EC0FF0F9EC2EF01FEF29F087C32AF19C
:1062500088C32BF189C32CF18AC32DF18BC32EF196
:106260008CC32FF18DC330F18EC331F190C332F165
:1062700091C333F10101296B7BEC36F0F2EC35F080
:10628000880E046F130E056F000E066F000E076F69
:1062900037EC35F0000E046F040E056F000E066F2C
:1062A000000E076F43EC35F00101E80E046F800E1D
:1062B000056F000E066F000E076F63EC35F0060EDB
:1062C0000C6E00C10BF0A6EC0BF0070E0C6E01C1BA
:1062D0000BF0A6EC0BF0080E0C6E02C10BF0A6EC56
:1062E0000BF0090E0C6E03C10BF0A6EC0BF00401D1
:1062F0007A0E826F38EC0FF004012C0E826F38ECAE
:106300000FF00401380E826F38EC0FF004012C0EF0
:10631000826F38EC0FF08BEC2FF01FEF29F007A8FD
:1063200003EF32F00101800E006F1A0E016F060EAE
:10633000026F000E036F4BC104F14CC105F14DC15A
:1063400006F14EC107F132EC35F003BF4AEF32F0EF
:10635000ADEC33F04BC100F14CC101F14DC102F184
:106360004EC103F107823FEC34F018C104F119C1AA
:1063700005F11AC106F11BC107F1F80E006FCD0E31
:10638000016F660E026F030E036F32EC35F00E0ED6
:106390000C6E00C10BF0A6EC0BF00F0E0C6E01C1E1
:1063A0000BF0A6EC0BF0100E0C6E02C10BF0A6EC7D
:1063B0000BF0110E0C6E03C10BF0A6EC0BF0078472
:1063C00001012DEC36F057C100F158C101F10794DD
:1063D0000A0E0C6E00C10BF0A6EC0BF00B0E0C6E4F
:1063E00001C10BF0A6EC0BF00C0E0C6E02C10BF011
:1063F000A6EC0BF00D0E0C6E03C10BF0A6EC0BF02F
:1064000007984AEF32F007AA4AEF32F007840101F9
:106410002DEC36F057C100F158C101F10794060E7A
:106420000C6E00C10BF0A6EC0BF0070E0C6E01C158
:106430000BF0A6EC0BF0080E0C6E02C10BF0A6ECF4
:106440000BF0090E0C6E03C10BF0A6EC0BF00784E9
:1064500062C100F163C101F164C102F165C103F1E0
:106460000794120E0C6E00C10BF0A6EC0BF0130E8D
:106470000C6E01C10BF0A6EC0BF0140E0C6E02C1F9
:106480000BF0A6EC0BF0150E0C6E03C10BF0A6EC96
:106490000BF0079A0401805181197F0B0DE09EA833
:1064A000FED714EE00F081517F0BE126E750812BDF
:1064B0000F01AD6E4AEF32F005012F51010A13E0D2
:1064C00081AA73EF32F005012F51000A0AE00FB8DC
:1064D00073EF32F00501306773EF32F00FB873EFEE
:1064E00032F0EAEF3FF081B888EF32F07CEC38F020
:1064F00005012F51020A02E088EF32F0602F88EF89
:1065000032F05FC560F50501010E306F3C0E316F52
:1065100084EF0EF006013251385D3351D8A0010FDF
:10652000395D800BD8A499EF32F032C638F633C605
:1065300039F6120006013251365D3351D8A0010FF1
:10654000375D800BD8B4A9EF32F032C636F633C6C9
:1065500037F6120007841AC632F61BC633F61CC67D
:1065600038F61DC639F68AEC32F01EC632F61FC662
:1065700033F68AEC32F020C632F621C633F68AECC6
:1065800032F01AC632F61BC633F61CC636F61DC6E6
:1065900037F69AEC32F01EC632F61FC633F69AEC86
:1065A00032F020C632F621C633F69AEC32F038517A
:1065B000365F3951D8A03929375F2DEC36F036C611
:1065C00000F137C601F139EC36F000C13AF601C1ED
:1065D0003BF622C632F623C633F624C638F625C665
:1065E00039F68AEC32F026C632F627C633F68AEC44
:1065F00032F028C632F629C633F68AEC32F022C6CB
:1066000032F623C633F624C636F625C637F69AEC9C
:1066100032F026C632F627C633F69AEC32F028C698
:1066200032F629C633F69AEC32F03851365F3951DA
:10663000D8A03929375F2DEC36F036C600F137C6C1
:1066400001F139EC36F000C13CF601C13DF62AC635
:1066500032F62BC633F62CC638F62DC639F68AEC40
:1066600032F02EC632F62FC633F68AEC32F030C640
:1066700032F631C633F68AEC32F02AC632F62BC631
:1066800033F62CC636F62DC637F69AEC32F02EC607
:1066900032F62FC633F69AEC32F030C632F631C6F7
:1066A00033F69AEC32F03851365F3951D8A0392997
:1066B000375F2DEC36F036C600F137C601F139EC04
:1066C00036F000C13EF601C13FF63AC632F63BC68F
:1066D00033F63CC636F63DC637F69AEC32F03EC687
:1066E00032F63FC633F69AEC32F00794120018C126
:1066F00000F119C101F11AC102F11BC103F1000E31
:10670000046F000E056F010E066F000E076F63EC3D
:1067100035F029A1A2EF33F02051D8B4A2EF33F025
:1067200018C100F119C101F11AC102F11BC103F135
:10673000000E046F000E056F0A0E066F000E076F45
:1067400063EC35F0120001010451001305510113EF
:10675000065102130751031312000101186B196B44
:106760001A6B1B6B12002AC182F40401300E8227BF
:1067700038EC0FF02BC182F40401300E822738EC84
:106780000FF02CC182F40401300E822738EC0FF098
:106790002DC182F40401300E822738EC0FF02EC197
:1067A00082F40401300E822738EC0FF02FC182F4FE
:1067B0000401300E822738EC0FF030C182F404015E
:1067C000300E822738EC0FF031C182F40401300E14
:1067D000822738EC0FF032C182F40401300E822798
:1067E00038EC0FF033C182F40401300E822738EC0C
:1067F0000FF012002FC182F40401300E822738EC12
:106800000FF030C182F40401300E822738EC0FF013
:1068100031C182F40401300E822738EC0FF032C10E
:1068200082F40401300E822738EC0FF033C182F479
:106830000401300E822738EC0FF01200060E1D6E98
:10684000060E1E6E060E1F6E1D2E24EF34F01E2E39
:1068500024EF34F01F2E24EF34F08B84020E1D6ED3
:10686000020E1E6E020E1F6E1D2E34EF34F01E2E11
:1068700034EF34F01F2E34EF34F08B94120001010A
:10688000005305E1015303E1025301E1002B02EC47
:1068900035F02DEC36F03951006F3A51016F420E50
:1068A000046F4B0E056F000E066F000E076F43EC72
:1068B00035F000C104F101C105F102C106F103C1C7
:1068C00007F118C100F119C101F11AC102F11BC190
:1068D00003F107B270EF34F037EC35F072EF34F0BB
:1068E00032EC35F000C118F101C119F102C11AF101
:1068F00003C11BF112002DEC36F059C100F15AC151
:1069000001F1060EBDEC0BF0E8CF04F1070EBDEC73
:106910000BF0E8CF05F1080EBDEC0BF0E8CF06F167
:10692000090EBDEC0BF0E8CF07F132EC35F000C1F9
:1069300024F101C125F102C126F103C127F1290E7D
:10694000046F000E056F000E066F000E076F43EC1C
:1069500035F0EE0E046F430E056F000E066F000E4D
:10696000076F37EC35F024C104F125C105F126C1CC
:1069700006F127C107F143EC35F000C11CF101C15C
:106980001DF102C11EF103C11FF1120EBDEC0BF08F
:10699000E8CF04F1130EBDEC0BF0E8CF05F1140EB7
:1069A000BDEC0BF0E8CF06F1150EBDEC0BF0E8CF17
:1069B00007F10D0E006F000E016F000E026F000E4A
:1069C000036F43EC35F0180E046F000E056F000ED8
:1069D000066F000E076F63EC35F01CC104F11DC19A
:1069E00005F11EC106F11FC107F137EC35F06A0E43
:1069F000046F2A0E056F000E066F000E076F32EC53
:106A000035F01200BF0EFA6E200E3A6F396BD89037
:106A10000037013702370337D8B013EF35F03A2F7C
:106A200008EF35F039073A070353D8B412000331A1
:106A3000070B80093F6F03390F0B010F396F80EC93
:106A40005FF0406F390580EC5FF0405D405F396B6F
:106A50003F33D8B0392739333FA928EF35F04051BB
:106A600039271200010152EC36F0D8B012000101B2
:106A700003510719346F15EC36F0D89007510319FC
:106A800034AF800F12000101346B39EC36F0D8A01E
:106A90004FEC36F0D8B0120024EC36F02DEC36F086
:106AA0001F0E366F65EC36F00B35D8B015EC36F0AE
:106AB000D8A00335D8B01200362F52EF35F034B1DC
:106AC0003CEC36F012000101346B04510511061143
:106AD00007110008D8A039EC36F0D8A04FEC36F0FA
:106AE000D8B01200086B096B0A6B0B6B65EC36F0C3
:106AF0001F0E366F65EC36F007510B5DD8A48DEF95
:106B000035F006510A5DD8A48DEF35F00551095DC9
:106B1000D8A48DEF35F00451085DD8A0A0EF35F072
:106B20000451085F0551D8A0053D095F0651D8A062
:106B3000063D0A5F0751D8A0073D0B5FD890008142
:106B4000362F7AEF35F034B13CEC36F0346B39EC5B
:106B500036F0D89069EC36F007510B5DD8A4BDEF44
:106B600035F006510A5DD8A4BDEF35F00551095D39
:106B7000D8A4BDEF35F00451085DD8A0CCEF35F0B6
:106B8000003FCCEF35F0013FCCEF35F0023FCCEFCA
:106B900035F0032BD8B4120034B13CEC36F01200BF
:106BA0000101346B39EC36F0D8B012006EEC36F0DF
:106BB000200E366F003701370237033711EE33F0FE
:106BC0000A0E376FE7360A0EE75CD8B0E76EE5527B
:106BD000372FE2EF35F0362FDAEF35F034B1298177
:106BE000D890120001010A0E346F200E366F11EE9C
:106BF00029F03451376F0A0ED890E652D8B0E72604
:106C0000E732372FFDEF35F0033302330133003322
:106C1000362FF7EF35F0E750FF0FD8A00335D8B087
:106C2000120029B13CEC36F0120004510027055146
:106C3000D8B0053D01270651D8B0063D02270751BF
:106C4000D8B0073D032712000051086F0151096FAA
:106C500002510A6F03510B6F12000101006B016BAF
:106C6000026B036B12000101046B056B066B076B73
:106C700012000335D8A012000351800B001F011F22
:106C8000021F031F003F4CEF36F0013F4CEF36F080
:106C9000023F4CEF36F0032B342B0325120007354F
:106CA000D8A012000751800B041F051F061F071FE5
:106CB000043F62EF36F0053F62EF36F0063F62EFC9
:106CC00036F0072B342B0725120000370137023727
:106CD0000337083709370A370B3712000101296BD0
:106CE0002A6B2B6B2C6B2D6B2E6B2F6B306B316BE0
:106CF000326B336B120001012A510F0B2A6F2B519B
:106D00000F0B2B6F2C510F0B2C6F2D510F0B2D6F69
:106D10002E510F0B2E6F2F510F0B2F6F30510F0B6A
:106D2000306F31510F0B316F32510F0B326F3351C6
:106D30000F0B336F1200899C000EC76E200EC66EBB
:106D40009E96C69EC50EC96EFF0E9EB602D0E82E58
:106D5000FCD79E96C69E000EC96EFF0E9EB602D050
:106D6000E82EFCD7C9CF00F69E96C69E000EC96ECF
:106D7000FF0E9EB602D0E82EFCD7C9CF01F6898C53
:106D80001200000EC76E200EC66E899C9E96C69E8F
:106D9000C80EC96EFF0E9EB602D0E82EFCD79E9696
:106DA000C69E000EC96EFF0E9EB602D0E82EFCD71E
:106DB000C9CF02F69E96C69E000EC96EFF0E9EB605
:106DC00002D0E82EFCD7C9CF03F69E96C69E000ED1
:106DD000C96EFF0E9EB602D0E82EFCD7C9CF0AF6C8
:106DE0009E96C69E000EC96EFF0E9EB602D0E82E7D
:106DF000FCD7C9CF0BF69E96C69E000EC96EFF0E3D
:106E00009EB602D0E82EFCD7C9CF12F69E96C69E3B
:106E1000000EC96EFF0E9EB602D0E82EFCD7C9CF79
:106E200013F6898C1200000EC76E200EC66E899C68
:106E30009E96C69EE80EC96EFF0E9EB602D0E82E44
:106E4000FCD79E96C69E000EC96EFF0E9EB602D05F
:106E5000E82EFCD7C9CF1AF69E96C69E000EC96EC4
:106E6000FF0E9EB602D0E82EFCD7C9CF1BF69E9629
:106E7000C69E000EC96EFF0E9EB602D0E82EFCD74D
:106E8000C9CF22F69E96C69E000EC96EFF0E9EB614
:106E900002D0E82EFCD7C9CF23F69E96C69E000EE0
:106EA000C96EFF0E9EB602D0E82EFCD7C9CF2AF6D7
:106EB0009E96C69E000EC96EFF0E9EB602D0E82EAC
:106EC000FCD7C9CF2BF6898C1200000EC76E200E9E
:106ED000C66E899C9E96C69E240EC96EFF0E9EB6F7
:106EE00002D0E82EFCD79E96C69EE40EC96EFF0E19
:106EF0009EB602D0E82EFCD7898C899C9E96C69EB1
:106F0000200EC96EFF0E9EB602D0E82EFCD79E96CC
:106F1000C69E5F0EC96EFF0E9EB602D0E82EFCD74D
:106F2000898C899C9E96C69E210EC96EFF0E9EB6C8
:106F300002D0E82EFCD79E96C69EC00EC96EFF0EEC
:106F40009EB602D0E82EFCD7898C899C9E96C69E60
:106F5000260EC96EFF0E9EB602D0E82EFCD79E9676
:106F6000C69E000EC96EFF0E9EB602D0E82EFCD75C
:106F7000898C120010A806D08994000EC76E220ECC
:106F8000C66E05D08984000EC76E220EC66E050E31
:106F9000E82EFED7120010A802D0898401D089946F
:106FA000050EE82EFED71200BAEC37F09E96C69E6C
:106FB000000EC96EFF0E9EB602D0E82EFCD79E963C
:106FC000C69E000EC96EFF0E9EB602D0E82EFCD7FC
:106FD000C9CFAFF59E96C69E000EC96EFF0E9EB637
:106FE00002D0E82EFCD7C9CFB0F59E96C69E000E03
:106FF000C96EFF0E9EB602D0E82EFCD7C9CFB1F500
:107000009E96C69E000EC96EFF0E9EB602D0E82E5A
:10701000FCD7C9CFB2F59E96C69E000EC96EFF0E74
:107020009EB602D0E82EFCD7C9CFB3F59E96C69E79
:10703000000EC96EFF0E9EB602D0E82EFCD7C9CF57
:10704000B4F59E96C69E000EC96EFF0E9EB602D087
:10705000E82EFCD7C9CFB5F5CBEC37F01200BAEC6F
:1070600037F09E96C69E800EC96EFF0E9EB602D069
:10707000E82EFCD79E96C69EAFC5C9FFFF0E9EB6F2
:1070800002D0E82EFCD79E96C69EB0C5C9FFFF0E63
:107090009EB602D0E82EFCD79E96C69EB1C5C9FF0B
:1070A000FF0E9EB602D0E82EFCD79E96C69EB2C5B5
:1070B000C9FFFF0E9EB602D0E82EFCD79E96C69E54
:1070C000B3C5C9FFFF0E9EB602D0E82EFCD79E9630
:1070D000C69EB4C5C9FFFF0E9EB602D0E82EFCD7EF
:1070E0009E96C69EB5C5C9FFFF0E9EB602D0E82E7D
:1070F000FCD7CBEC37F01200BAEC37F09E96C69E68
:10710000070EC96EFF0E9EB602D0E82EFCD79E96E3
:10711000C69E000EC96EFF0E9EB602D0E82EFCD7AA
:10712000C9CFAFF59E96C69E000EC96EFF0E9EB6E5
:1071300002D0E82EFCD7C9CFB0F59E96C69E000EB1
:10714000C96EFF0E9EB602D0E82EFCD7C9CFB1F5AE
:107150009E96C69E000EC96EFF0E9EB602D0E82E09
:10716000FCD7C9CFB2F5CBEC37F0BAEC37F09E962E
:10717000C69E21C0C9FFFF0E9EB602D0E82EFCD7E6
:107180009E96C69E000EC96EFF0E9EB602D0E82ED9
:10719000FCD7C9CFB6F5CBEC37F01200BAEC37F01C
:1071A0009E96C69E870EC96EFF0E9EB602D0E82E32
:1071B000FCD79E96C69EAFC5C9FFFF0E9EB602D0F5
:1071C000E82EFCD79E96C69EB0C5C9FFFF0E9EB6A0
:1071D00002D0E82EFCD79E96C69EB1C5C9FFFF0E11
:1071E0009EB602D0E82EFCD79E96C69EB2C5C9FFB9
:1071F000FF0E9EB602D0E82EFCD7CBEC37F0BAECEF
:1072000037F09E96C69E22C0C9FFFF0E9EB602D0E2
:10721000E82EFCD79E96C69EB6C5C9FFFF0E9EB649
:1072200002D0E82EFCD7CBEC37F01200BAEC37F0E6
:107230009E96C69E870EC96EFF0E9EB602D0E82EA1
:10724000FCD79E96C69E000EC96EFF0E9EB602D05B
:10725000E82EFCD79E96C69E800EC96EFF0E9EB687
:1072600002D0E82EFCD79E96C69E800EC96EFF0EF9
:107270009EB602D0E82EFCD79E96C69E800EC96EA2
:10728000FF0E9EB602D0E82EFCD7CBEC37F01200F2
:10729000BAEC37F09E96C69E870EC96EFF0E9EB65C
:1072A00002D0E82EFCD79E96C69E000EC96EFF0E39
:1072B0009EB602D0E82EFCD79E96C69E000EC96EE2
:1072C000FF0E9EB602D0E82EFCD79E96C69E800E7C
:1072D000C96EFF0E9EB602D0E82EFCD79E96C69EC3
:1072E000800EC96EFF0E9EB602D0E82EFCD7CBEC06
:1072F00037F0120010A82DD0BAEC37F09E96C69E3B
:1073000022C0C9FFFF0E9EB602D0E82EFCD79E9683
:10731000C69E450EC96EFF0E9EB602D0E82EFCD763
:10732000CBEC37F0BAEC37F09E96C69E8F0EC96E46
:10733000FF0E9EB602D0E82EFCD79E96C69E000E8B
:10734000C96EFF0E9EB602D0E82EFCD7CBEC37F00C
:107350001200BAEC37F09E96C69E22C0C9FFFF0EFF
:107360009EB602D0E82EFCD79E96C69E010EC96E30
:10737000FF0E9EB602D0E82EFCD7CBEC37F0BAEC6D
:1073800037F09E96C69E910EC96EFF0E9EB602D035
:10739000E82EFCD79E96C69EA50EC96EFF0E9EB621
:1073A00002D0E82EFCD7CBEC37F01200BAEC37F065
:1073B0009E96C69E22C0C9FFFF0E9EB602D0E82E42
:1073C000FCD79E96C69E810EC96EFF0E9EB602D059
:1073D000E82EFCD7CBEC37F01200BAEC37F09E96D3
:1073E000C69E22C0C9FFFF0E9EB602D0E82EFCD773
:1073F0009E96C69E010EC96EFF0E9EB602D0E82E66
:10740000FCD7CBEC37F01200BAEC37F09E96C69E54
:10741000910EC96EFF0E9EB602D0E82EFCD79E9646
:10742000C69EA50EC96EFF0E9EB602D0E82EFCD7F2
:10743000CBEC37F01200BAEC37F09E96C69E910E58
:10744000C96EFF0E9EB602D0E82EFCD79E96C69E51
:10745000000EC96EFF0E9EB602D0E82EFCD7CBEC14
:1074600037F012000501256B266B276B286B899A74
:10747000400EC76E200EC66E9E96C69E030EC96E47
:10748000FF0E9EB602D0E82EFCD79E96C69E27C55C
:10749000C9FFFF0E9EB602D0E82EFCD79E96C69E70
:1074A00026C5C9FFFF0E9EB602D0E82EFCD79E96D9
:1074B000C69E25C5C9FFFF0E9EB602D0E82EFCD79A
:1074C0009E96C69EC952FF0E9EB602D0E82EFCD7ED
:1074D000898A0F01C950FF0A01E1120005012E51EE
:1074E000130A05E005012E51170A0CE012000501F0
:1074F000E00E256FFF0E266F0F0E276F000E286F10
:107500008BEF3AF00501E00E256FFF0E266FFF0EA0
:10751000276F000E286F899A400EC76E200EC66E28
:107520009E96C69E030EC96EFF0E9EB602D0E82E32
:10753000FCD79E96C69E27C5C9FFFF0E9EB602D0F9
:10754000E82EFCD79E96C69E26C5C9FFFF0E9EB6A6
:1075500002D0E82EFCD79E96C69E25C5C9FFFF0E19
:107560009EB602D0E82EFCD79E96C69EC952FF0E4C
:107570009EB602D0E82EFCD7898A0F01C950FF0AB7
:107580001DE005012E51130A05E005012E51170AD1
:107590000BE012000501000E256F000E266F100E85
:1075A000276F000E286F12000501000E256F000ED8
:1075B000266F000E276F010E286F12000501256B44
:1075C000266B276B286B05012E51130A05E0050178
:1075D0002E51170A0CE012000501000E216F000E5B
:1075E000226F080E236F000E246F00EF3BF00501A1
:1075F000000E216F000E226F800E236F000E246F8D
:1076000021C500F122C501F123C502F124C503F112
:1076100025C504F126C505F127C506F128C507F1E2
:10762000A3EC33F000C125F501C126F502C127F511
:1076300003C128F5899A400EC76E200EC66E9E962D
:10764000C69E030EC96EFF0E9EB602D0E82EFCD772
:107650009E96C69E27C5C9FFFF0E9EB602D0E82E95
:10766000FCD79E96C69E26C5C9FFFF0E9EB602D0C9
:10767000E82EFCD79E96C69E25C5C9FFFF0E9EB676
:1076800002D0E82EFCD79E96C69EC952FF0E9EB62B
:1076900002D0E82EFCD7898AC950FF0A08E104C14C
:1076A00025F505C126F506C127F507C128F5D890AF
:1076B000050124332333223321332151E00B216F81
:1076C00021676AEF3BF022676AEF3BF023676AEFBE
:1076D0003BF0246700EF3BF00501200E2527E86A08
:1076E0002623E86A2723E86A28231200E86A0501AE
:1076F0002E51130A06E005012E51170A0BE0020E67
:10770000120005012851000A03E12751F00B07E0A0
:10771000010E120005012851000A01E0010E1200BD
:1077200029C500F12AC501F12BC502F12CC503F1D1
:1077300025C504F126C505F127C506F128C507F1C1
:1077400032EC35F003BF120076EC3BF0D8A408EF22
:107750003CF0899A400EC76E200EC66E9E96C69E5D
:10776000060EC96EFF0E9EB602D0E82EFCD7898A9F
:10777000899A9E96C69E020EC96EFF0E9EB602D0D4
:10778000E82EFCD79E96C69E27C5C9FFFF0E9EB663
:1077900002D0E82EFCD79E96C69E26C5C9FFFF0ED6
:1077A0009EB602D0E82EFCD79E96C69E25C5C9FF80
:1077B000FF0E9EB602D0E82EFCD79E96C69E000E07
:1077C000C96EFF0E9EB602D0E82EFCD7898A899A30
:1077D0009E96C69E050EC96EFF0E9EB602D0E82E7E
:1077E000FCD79E96C69EC952FF0E9EB602D0E82ECA
:1077F000FCD7C9B0F1EF3BF0898A0501200E25279F
:10780000E86A2623E86A2723E86A282390EF3BF0FA
:107810001200899A400EC76E200EC66E9E96C69EB6
:10782000060EC96EFF0E9EB602D0E82EFCD7898ADE
:10783000899A9E96C69EC70EC96EFF0E9EB602D04E
:10784000E82EFCD7898A0501256B266B276B286BF0
:107850001200899A400EC76E200EC66E9E96C69E76
:10786000050EC96EFF0E9EB602D0E82EFCD79E967E
:10787000C69EC952FF0E9EB602D0E82EFCD7C9CFD5
:1078800037F5898A1200899A400EC76E200EC66E9F
:107890009E96C69EB90EC96EFF0E9EB602D0E82E09
:1078A000FCD7898A1200899A400EC76E200EC66ED8
:1078B0009E96C69EAB0EC96EFF0E9EB602D0E82EF7
:1078C000FCD7898AFF0EE82EFED7120076EC3BF03B
:1078D000D8A41200899A400EC76E200EC66E9E96DE
:1078E000C69E030EC96EFF0E9EB602D0E82EFCD7D0
:1078F0009E96C69E27C5C9FFFF0E9EB602D0E82EF3
:10790000FCD79E96C69E26C5C9FFFF0E9EB602D026
:10791000E82EFCD79E96C69E25C5C9FFFF0E9EB6D3
:1079200002D0E82EFCD79E96C69EC952FF0E9EB688
:1079300002D0E82EFCD7898A0F01C950FF0AD8A4CB
:107940005DEF3FF00501FE0E376FD4EC37F0AFC5A9
:1079500038F5B0C539F5B1C53AF5B2C53BF5B3C593
:107960003CF5B4C53DF5B5C53EF50784B6C166F135
:10797000B7C167F1B8C168F1B9C169F14BC14FF145
:107980004CC150F14DC151F14EC152F157C159F1A5
:1079900058C15AF149EC29F000C13FF501C140F549
:1079A00002C141F503C142F505016167DFEF3CF01B
:1079B0006267DFEF3CF06367DFEF3CF06467E3EFA3
:1079C0003CF0F0EF3CF061C504F162C505F163C520
:1079D00006F164C507F132EC35F003BF5DEF3FF00F
:1079E00059C143F55AC144F5B9C545F5BAC546F57F
:1079F000AAEC32F036C649F537C64AF506014067AB
:107A000009EF3DF0416709EF3DF0426709EF3DF0B6
:107A100043670DEF3DF01EEF3DF02DEC36F033ECFB
:107A200036F036C600F137C601F140C604F141C652
:107A300005F132EC35F003AF5DEF3FF00101036B70
:107A4000026B1AC600F11BC601F101AF2CEF3DF02D
:107A5000FF0E026FFF0E036F0101076B066B1CC662
:107A600004F11DC605F105AF3AEF3DF0FF0E066FBC
:107A7000FF0E076F37EC35F00101076B066B1EC672
:107A800004F11FC605F105AF4AEF3DF0FF0E066F8A
:107A9000FF0E076F37EC35F00101076B066B20C650
:107AA00004F121C605F105AF5AEF3DF0FF0E066F58
:107AB000FF0E076F37EC35F0D89001010333023326
:107AC00001330033D8900101033302330133003313
:107AD00000C14BF501C14CF50101036B026B22C6DD
:107AE00000F123C601F101AF7AEF3DF0FF0E026F06
:107AF000FF0E036F0101076B066B24C604F125C658
:107B000005F105AF88EF3DF0FF0E066FFF0E076F22
:107B100037EC35F00101076B066B26C604F127C66A
:107B200005F105AF98EF3DF0FF0E066FFF0E076FF2
:107B300037EC35F00101076B066B28C604F129C646
:107B400005F105AFA8EF3DF0FF0E066FFF0E076FC2
:107B500037EC35F0D89001010333023301330033A1
:107B6000D8900101033302330133003300C14DF5D6
:107B700001C14EF50101036B026B2AC600F12BC651
:107B800001F101AFC8EF3DF0FF0E026FFF0E036F72
:107B90000101076B066B2CC604F12DC605F105AF7C
:107BA000D6EF3DF0FF0E066FFF0E076F37EC35F096
:107BB0000101076B066B2EC604F12FC605F105AF58
:107BC000E6EF3DF0FF0E066FFF0E076F37EC35F066
:107BD0000101076B066B30C604F131C605F105AF34
:107BE000F6EF3DF0FF0E066FFF0E076F37EC35F036
:107BF000D89001010333023301330033D8900101DF
:107C0000033302330133003300C14FF501C150F596
:107C10000101036B026B02C600F103C601F101AF63
:107C200016EF3EF0FF0E026FFF0E036F0101076BB0
:107C3000066B04C604F105C605F105AF24EF3EF05E
:107C4000FF0E066FFF0E076F37EC35F00101076B73
:107C5000066B06C604F107C605F105AF34EF3EF02A
:107C6000FF0E066FFF0E076F37EC35F00101076B53
:107C7000066B08C604F109C605F105AF44EF3EF0F6
:107C8000FF0E066FFF0E076F37EC35F0D89001013D
:107C90000333023301330033D8900101033302333D
:107CA0000133003300C151F501C152F50101036BED
:107CB000026B0AC600F10BC601F101AF64EF3EF0A2
:107CC000FF0E026FFF0E036F0101076B066B0CC600
:107CD00004F10DC605F105AF72EF3EF0FF0E066F21
:107CE000FF0E076F37EC35F00101076B066B0EC610
:107CF00004F10FC605F105AF82EF3EF0FF0E066FEF
:107D0000FF0E076F37EC35F00101076B066B10C6ED
:107D100004F111C605F105AF92EF3EF0FF0E066FBC
:107D2000FF0E076F37EC35F0D890010103330233B3
:107D300001330033D89001010333023301330033A0
:107D400000C153F501C154F50101036B026B12C66A
:107D500000F113C601F101AFB2EF3EF0FF0E026F6A
:107D6000FF0E036F0101076B066B14C604F115C605
:107D700005F105AFC0EF3EF0FF0E066FFF0E076F77
:107D800037EC35F00101076B066B16C604F117C618
:107D900005F105AFD0EF3EF0FF0E066FFF0E076F47
:107DA00037EC35F00101076B066B18C604F119C6F4
:107DB00005F105AFE0EF3EF0FF0E066FFF0E076F17
:107DC00037EC35F0D890010103330233013300332F
:107DD000D8900101033302330133003300C155F55C
:107DE00001C156F507940501210E326F899A400EA4
:107DF000C76E200EC66E9E96C69E060EC96EFF0EFC
:107E00009EB602D0E82EFCD7898A899A9E96C69E95
:107E1000020EC96EFF0E9EB602D0E82EFCD79E96CB
:107E2000C69E27C5C9FFFF0E9EB602D0E82EFCD71E
:107E30009E96C69E26C5C9FFFF0E9EB602D0E82EAE
:107E4000FCD79E96C69E25C5C9FFFF0E9EB602D0E2
:107E5000E82EFCD725EE37F0322F02D03BEF3FF073
:107E60009E96C69EDECFC9FFFF0E9EB602D0E82EBC
:107E7000FCD72CEF3FF0898A899A9E96C69E050E04
:107E8000C96EFF0E9EB602D0E82EFCD79E96C69E07
:107E9000C952FF0E9EB602D0E82EFCD7C9B046EFFD
:107EA0003FF0898A0501200E2527E86A2623E86A23
:107EB0002723E86A28231EEC34F0120021C500F1C4
:107EC00022C501F123C502F124C503F1899A400EB0
:107ED000C76E200EC66E9E96C69E0B0EC96EFF0E16
:107EE0009EB602D0E82EFCD79E96C69E02C1C9FF60
:107EF000FF0E9EB602D0E82EFCD79E96C69E01C10C
:107F0000C9FFFF0E9EB602D0E82EFCD79E96C69EF5
:107F100000C1C9FFFF0E9EB602D0E82EFCD79E9688
:107F2000C69EC952FF0E9EB602D0E82EFCD725EEA3
:107F300037F00501200E326F9E96C69EC952FF0E85
:107F40009EB602D0E82EFCD7C9CFDEFF322F9CEFC1
:107F50003FF0898A1200899A400EC76E200EC66EC5
:107F60009E96C69E900EC96EFF0E9EB602D0E82E5B
:107F7000FCD79E96C69E000EC96EFF0E9EB602D01E
:107F8000E82EFCD79E96C69E000EC96EFF0E9EB6CA
:107F900002D0E82EFCD79E96C69E000EC96EFF0E3C
:107FA0009EB602D0E82EFCD79E96C69EC952FF0E02
:107FB0009EB602D0E82EFCD7C9CF2DF59E96C69E60
:107FC000C952FF0E9EB602D0E82EFCD7C9CF2EF5BF
:107FD000898A12001EEC34F0B9C5E8FFD70802E325
:107FE0001EEC34F0B9C5E8FFC80802E31EEC34F01B
:107FF000B9C5E8FFB90802E31EEC34F0B9C5E8FFE3
:10800000AA0802E31EEC34F0B9C5E8FF9B0802E3BE
:108010001EEC34F07CEC38F043EC3CF0F29CF29E29
:108020008B94C69AC290898C9482948C720ED36E73
:10803000D3A4FED789968A909390FF0EE8CF00F0E4
:10804000E82EFED7002EFCD78150F294F29A9E9033
:108050009D909E929D92F298F292F290F286F28E0C
:048060000300FF001A
:10BF0000E844F926000C160C2B0C3F0C520C640C68
:10BF1000760C860C960CA50CB30CC10CCF0CDC0C6B
:06BF2000E80CF40C000C1B
:00000001FF
